:100000000C9490030C94AD030C94AD030C94A928AC
:100010000C945F120C94AD030C94AD030C94AD03DF
:100020000C94AD030C94F2140C94AD030C941F16B5
:100030000C94AD030C94AD030C94AD030C94AD0380
:100040000C94AD030C94AD030C940D120C94C811D8
:100050000C94AD030C94AD030C94AD030C94AD0360
:100060000C94AD030C94AD038F1A8F1A8F1AA61A35
:10007000BB1AC41ACD1AD61ADF1AF61A021B0B1BAA
:10008000141B1D1B2F1B431B551B6B1B7D1B861B32
:100090008F1B981BA31B084AD73B3BCE016E84BC29
:1000A000BFFDC12F3D6C74319ABD56833DDA3D00D2
:1000B000C77F11BED9E4BB4C3E916BAAAABE00001B
:1000C00000803F05A84CCDB2D44EB93836A9020CF9
:1000D00050B9918688083CA6AAAA2ABE00000080D2
:1000E0003F3E0D0A002C0057506F733A002C002C35
:1000F0004D506F733A003C436865636B003C416C44
:1001000061726D003C486F6D65003C486F6C640027
:100110003C52756E003C5175657565003C49646CD8
:1001200065000D0A003D00244E005D0D0A002046CA
:1001300000205400204D3800204D3900204D35005E
:10014000204D3400204D3300204D3200204D310031
:10015000204D3000204739340020473933002047F4
:1001600039310020473930002047323100204732F2
:1001700030002047313900204731380020473137DF
:10018000002047005B473830005B4733005B473255
:10019000005B4731005B4730005D0D0A002C005BBF
:1001A0004739323A005D0D0A002C0033303A0032F4
:1001B000383A0035393A0035383A0035373A0035A3
:1001C000363A0035353A0035343A005B470020288E
:1001D000686F6D696E672070756C6C2D6F66662C2C
:1001E000206D6D290D0A002028686F6D696E6720EB
:1001F0006465626F756E63652C206D736563290D90
:100200000A2432323D002028686F6D696E672073C2
:1002100065656B2C206D6D2F6D696E290D0A24327A
:10022000313D002028686F6D696E672066656564E2
:100230002C206D6D2F6D696E290D0A2432303D0022
:10024000290D0A2431393D002028686F6D696E67D9
:100250002064697220696E76657274206D61736BBB
:100260002C20696E743A002028686F6D696E6720D3
:100270006379636C652C20626F6F6C290D0A2431E1
:10028000383D00202868617264206C696D69747360
:100290002C20626F6F6C290D0A2431373D00202815
:1002A000696E76657274207374657020656E616224
:1002B0006C652C20626F6F6C290D0A2431363D006D
:1002C00020286175746F2073746172742C20626FC2
:1002D0006F6C290D0A2431353D0020287265706F3E
:1002E000727420696E636865732C20626F6F6C296D
:1002F0000D0A2431343D0020286E2D646563696D3C
:10030000616C732C20696E74290D0A2431333D0011
:1003100020286E2D61726320636F72726563746949
:100320006F6E2C20696E74290D0A2431323D002035
:10033000286172632C206D6D2F7365676D656E7417
:10034000290D0A2431313D0020286A756E637469D5
:100350006F6E20646576696174696F6E2C206D6DB7
:10036000290D0A2431303D002028616363656C65E6
:10037000726174696F6E2C206D6D2F7365635E32D0
:10038000290D0A24393D00202873746570206964A2
:100390006C652064656C61792C206D736563290D33
:1003A0000A24383D00290D0A24373D0020287374A3
:1003B000657020706F727420696E76657274206D3E
:1003C00061736B2C20696E743A0020286465666145
:1003D000756C74207365656B2C206D6D2F6D696E67
:1003E000290D0A24363D00202864656661756C7409
:1003F00020666565642C206D6D2F6D696E290D0A70
:1004000024353D002028737465702070756C736509
:100410002C2075736563290D0A24343D0020287A49
:100420002C20737465702F6D6D290D0A24333D00E7
:100430002028792C20737465702F6D6D290D0A2486
:10044000323D002028782C20737465702F6D6D2943
:100450000D0A24313D0024303D00242420287669F3
:100460006577204772626C2073657474696E677378
:10047000290D0A24232028766965772023207061BE
:1004800072616D6574657273290D0A2447202876A0
:100490006965772070617273657220737461746529
:1004A000290D0A244E2028766965772073746172BD
:1004B00074757020626C6F636B73290D0A24783D2C
:1004C00076616C7565202873617665204772626C71
:1004D0002073657474696E67290D0A244E783D6C2B
:1004E000696E652028736176652073746172747516
:1004F0007020626C6F636B290D0A244320286368A7
:1005000065636B2067636F6465206D6F6465290D9B
:100510000A245820286B696C6C20616C61726D2014
:100520006C6F636B290D0A2448202872756E206851
:100530006F6D696E67206379636C65290D0A7E2093
:10054000286379636C65207374617274290D0A21C4
:1005500020286665656420686F6C64290D0A3F2059
:100560002863757272656E74207374617475732973
:100570000D0A6374726C2D7820287265736574207F
:100580004772626C290D0A000D0A4772626C2030B6
:100590002E3863205B27242720666F722068656CE5
:1005A000705D0D0A005D0D0A0044697361626C653F
:1005B0006400456E61626C65640043617574696FC7
:1005C0006E3A20556E6C6F636B6564002724482774
:1005D0007C2724582720746F20756E6C6F636B0026
:1005E000526573657420746F20636F6E74696E75E5
:1005F00065005B002E204D506F733F0D0A00416275
:100600006F727420647572696E67206379636C65BC
:100610000048617264206C696D697400414C4152FC
:100620004D3A20000D0A004C696E65206F766572A8
:10063000666C6F7700416C61726D206C6F636B004C
:1006400042757379206F7220717565756564004518
:100650004550524F4D2072656164206661696C2E71
:10066000205573696E672064656661756C747300EC
:1006700056616C7565203C203320757365630056A8
:10068000616C7565203C20302E30005365747469B0
:100690006E672064697361626C656400496E76619F
:1006A0006C69642073746174656D656E74004D6F60
:1006B00064616C2067726F75702076696F6C61740D
:1006C000696F6E00496E76616C696420726164695D
:1006D000757300556E737570706F727465642073F6
:1006E000746174656D656E740045787065637465DA
:1006F0006420636F6D6D616E64206C6574746572E7
:1007000000426164206E756D62657220666F726D65
:100710006174006572726F723A20006F6B0D0A008F
:1007200011241FBECFEFD8E0DEBFCDBF11E0A0E0A7
:10073000B1E0E4EDF7E602C005900D92A030B107FC
:10074000D9F716E0A0E0B1E001C01D92A73FB107C4
:10075000E1F70E94AF030C94E8330C9400000F9370
:100760001F930E9495110E94AB1C0E94F115789472
:1007700080E1ECEBF5E0DF011D928A95E9F781E07D
:100780008093BC058093BD0506E011E08091BC0517
:10079000882389F10E9408120E94CA240E942B110A
:1007A0000E94B7140E9459110E947D110E942026B8
:1007B0000E94C4150E94E3251092BC051092BE054C
:1007C0008091E406982F81FF02C01093CB058091A1
:1007D000BD05813021F494FF02C00093BD058091D6
:1007E000BD05863021F482E00E94502A04C0109298
:1007F000BD050E94FC120E949B120E946614C6CF87
:100800008091BE0584FD15C08091BE0580618093F6
:10081000BE050E945F110E9482118091BD05835028
:10082000833038F48091BE0580628093BE050E94BB
:10083000D8150895EF92FF920F931F93CF93DF93F4
:100840007B018C0120E030E040EA51E40E94AE32AE
:100850000E94AB300E944230EB010E94AD24C801DF
:10086000B70120E030E04AE754E40E94AE327B0159
:100870008C0182E390E0C89FB001C99F700DD89FA2
:10088000700D112480E090E00E946E309B01AC015D
:10089000C801B7010E94F42E0E94AB300E94423082
:1008A000DC01CB010E94992500E911E00EC00E94F5
:1008B0009B128091BC05882351F484EF91E0F801EC
:1008C0003197F1F70197D9F72197209781F7DF91B9
:1008D000CF911F910F91FF90EF9008954F925F92EB
:1008E0006F927F928F92AF92BF92CF92DF92EF92F0
:1008F000FF920F931F93DF93CF9300D000D0CDB71B
:10090000DEB72B013C0129833A834B835C838091C2
:10091000BD058730F9F00E949B128091BC058823A9
:10092000C9F40E94311D8823B1F7C301B2012981A6
:100930003A814B815C810E94C2208091BD05882351
:1009400019F482E08093BD058091CB05882311F0D6
:100950000E946F150F900F900F900F90CF91DF9125
:100960001F910F91FF90EF90DF90CF90BF90AF90CD
:100970008F907F906F905F904F9008952F923F924D
:100980004F925F926F927F928F929F92AF92BF929F
:10099000CF92DF92EF92FF920F931F9385E08093A7
:1009A000BD0580916B00817F80936B000E944F2872
:1009B0000E949B128091BC05882309F070C08CE0D6
:1009C000EFEBF5E0DF011D928A95E9F70E94E32540
:1009D0001092BD053091E506232F35FD02C06FEF63
:1009E00001C061E026FD03C0DD24DA9402C0DD24ED
:1009F000D39437FD03C0CC24CA9402C0CC24C39442
:100A0000E090F006F090F1060091F2061091F306E6
:100A1000772767FD7095872F972F0E947030A80168
:100A200097010E94AE321B012C016D2D772767FDC7
:100A30007095872F972F0E947030A80197010E9410
:100A4000AE323B014C016C2D772767FD7095872FE7
:100A5000972F0E947030A80197010E94AE327B014F
:100A60008C01A090EA06B090EB06C090EC06D09006
:100A7000ED06C201B101A401930188240E946E0415
:100A80000E946F150E94AD240E94E3258091E40628
:100A900083FF05C080916B008E6080936B001F9177
:100AA0000F91FF90EF90DF90CF90BF90AF909F900D
:100AB0008F907F906F905F904F903F902F90089510
:100AC0002F923F924F925F926F927F928F929F925E
:100AD000AF92BF92CF92DF92EF92FF920F931F934C
:100AE000DF93CF93CDB7DEB7CE54D0400FB6F89496
:100AF000DEBF0FBECDBF3C017EAF6DAF21965FAFB5
:100B00004EAF219722962FAF229723960FAF2397B0
:100B10002496EFAE24972896ACAEBDAECEAEDFAE37
:100B2000289729968FAE2997E22EFF24EE0CFF1C02
:100B3000EE0CFF1C4E0D5F1D5CAF4BAFDA012D902C
:100B40003D904D905C90FC01EE0DFF1DC201B10186
:100B500020813181428153810E94F52E69AB7AABAD
:100B60008BAB9CAB10E0000F111F000F111F2196E3
:100B7000EEADFFAD2197E00FF11FFAAFE9AFA08016
:100B8000B180C280D380F301E00FF11FC601B5012F
:100B900020813181428153810E94F52E6DA77EA76D
:100BA0008FA798AB24962FAD2497E22FF0E0EE0F9D
:100BB000FF1FEE0FFF1F6E0E7F1ED3018D919D91C3
:100BC0000D90BC91A02D8DAB9EABAFABB8AF2DAD52
:100BD0003EADE20FF31F60817181828193812DA967
:100BE0003EA94FA958AD0E94F42E69A77AA78BA7FA
:100BF0009CA7D201C101B0588DA39EA3AFA3B8A7F3
:100C0000A6019501505829A33AA34BA35CA34DAD6F
:100C10005EADE40EF51ED7016D917D918D919C9195
:100C200029A93AA94BA95CA90E94F42E3B014C01C9
:100C3000EDADFEAD0E0F1F1FD8016D917D918D9111
:100C40009C912DA53EA54FA558A90E94F42E5B01AD
:100C50006C016DA17EA18FA198A5A60195010E94AE
:100C6000AE327B018C0169A17AA18BA19CA1A40168
:100C700093010E94AE329B01AC01C801B7010E94F2
:100C8000F42E1B012C016DA17EA18FA198A5A401BA
:100C900093010E94AE327B018C0169A17AA18BA1E4
:100CA0009CA1A60195010E94AE329B01AC01C80136
:100CB000B7010E94F52E9B01AC01C201B1010E9457
:100CC000682F5B016C01A8968FADA897882399F0D7
:100CD000C601B50120E030E040E050E00E94DC3188
:100CE0008823ECF0C601B5012BED3FE049EC50E460
:100CF0000E94F42E12C0C601B50120E030E040E0B1
:100D000050E00E94CE2F181654F0C601B5012BED0D
:100D10003FE049EC50E40E94F52E5B016C01C601F6
:100D2000B501A7962CAD3DAD4EAD5FADA7970E9426
:100D3000AE3229A53AA54BA55CA50E94E9317B01FD
:100D40008C0120E030E040E050E00E94CE2F88236C
:100D500009F4D5C1C801B7012091D8063091D90650
:100D60004091DA065091DB060E94D52F0E94AB30ED
:100D70000E94423078A36F8F2996BFAD2997BB237D
:100D8000A1F080E090E00E946E309B01AC012896BB
:100D90006CAD7DAD8EAD9FAD28970E94AE3228968A
:100DA0006CAF7DAF8EAF9FAF28972F8D38A1B90163
:100DB00080E090E00E946E307B018C01C601B5019D
:100DC000A80197010E94D52F6B8F7C8F8D8F9E8FEE
:100DD00069A57AA58BA59CA5A80197010E94D52F8E
:100DE0006F8B788F898F9A8F6B8D7C8D8D8D9E8D7B
:100DF00020E030E040E05FEB0E94AE322B8D3C8D76
:100E00004D8D5E8D0E94AE3220E030E040E85FE321
:100E10000E94F52E6B8B7C8B8D8B9E8B24963FAD29
:100E20002497E32FF0E0EE0FFF1FEE0FFF1FCE0120
:100E30000196E80FF91F2DA93EA94FA958AD2083AF
:100E400031834283538341E050E05E874D876624BF
:100E50002296BFAD2297AB2FB0E0AA0FBB1FAA0FFF
:100E6000BB1FA80FB91F2B96BFAFAEAF2B97239612
:100E70003FAD2397232F30E0220F331F220F331F64
:100E8000280F391F2D963FAF2EAF2D972F96FFAF0E
:100E9000EEAF2F970EC1262D332727FD3095809179
:100EA000F60690E0281739070CF046C06DA17EA128
:100EB0008FA198A52B8D3C8D4D8D5E8D0E94AE32FD
:100EC0007B018C0169A17AA18BA19CA12B893C8912
:100ED0004D895E890E94AE329B01AC01C801B70109
:100EE0000E94F52E7B018C016DA17EA18FA198A59A
:100EF0002B893C894D895E890E94AE325B016C0171
:100F000069A17AA18BA19CA12B8D3C8D4D8D5E8D0D
:100F10000E94AE329B01AC01C601B5010E94F42EC5
:100F20006DA37EA38FA398A76394C701D80189A35B
:100F30009AA3ABA3BCA361C04D855E85BA0180E0D6
:100F400090E00E946E302B8D3C8D4D8D5E8D0E9409
:100F5000AE327B018C01C8010E94D22F6F87788B43
:100F6000898B9A8BB701C8010E9431333B014C0138
:100F7000ABADBCADED90FD900D911C9117FB1095A4
:100F800017F91095E9ADFAAD208031804280538089
:100F9000C801B7012F85388949895A890E94AE3224
:100FA0005B016C01C201B101A40193010E94AE3248
:100FB0009B01AC01C601B5010E94F52E6DA37EA375
:100FC0008FA398A7C801B701A40193010E94AE3274
:100FD0007B018C01C201B1012F85388949895A8969
:100FE0000E94AE329B01AC01C801B7010E94F42EF1
:100FF00069A37AA38BA39CA3662469A97AA98BA968
:101000009CA92DA13EA14FA158A50E94F52E2B967B
:10101000AEADBFAD2B976D937D938D939C9313973E
:101020006DA57EA58FA598A929A13AA14BA15CA188
:101030000E94F52E2D96EEADFFAD2D976083718346
:10104000828393832F96AEADBFAD2F976D917D9127
:101050008D919C912F89388D498D5A8D0E94F52E46
:101060002F96EEADFFAD2F976083718382839383BC
:1010700069817A818B819C812D813E814F81588548
:10108000E984FA840B851C852896ACACBDACCEAC4B
:10109000DFAC289729968FAC29970E946E04809127
:1010A000BC05882361F52D853E852F5F3F4F3E8728
:1010B0002D874D855E858F8D98A14817590708F4B7
:1010C000EACEADADBEAD6D917D918D919C911397A2
:1010D00014962D913D914D915C9117971896ED9036
:1010E000FD900D911C911B972896ACACBDACCEAC7D
:1010F000DFAC289729968FAC29970E946E04C25BBB
:10110000DF4F0FB6F894DEBF0FBECDBFCF91DF919A
:101110001F910F91FF90EF90DF90CF90BF90AF9015
:101120009F908F907F906F905F904F903F902F9007
:101130000895AF92BF92CF92DF92EF92FF920F93FA
:101140001F9359016A010E9470302091C1063091AD
:10115000C2064091C3065091C4060E94D52F6093E9
:10116000D8057093D9058093DA059093DB05C60105
:10117000B5010E9470302091C5063091C60640919D
:10118000C7065091C8060E94D52F6093DC05709366
:10119000DD058093DE059093DF05C801B7010E944D
:1011A00070302091C9063091CA064091CB0650910B
:1011B000CC060E94D52F6093E0057093E1058093E3
:1011C000E2059093E3051F910F91FF90EF90DF9060
:1011D000CF90BF90AF9008952F923F924F925F9221
:1011E0006F927F928F929F92AF92BF92CF92DF9237
:1011F000EF92FF920F931F93DF93CF93CDB7DEB79C
:10120000EF970FB6F894DEBF0FBECDBF4C018091B3
:10121000BD05863011F48CE0C8C719828CE0FE0150
:101220003696DF01482F1D924A95E9F7FE01729626
:10123000DF011D928A95E9F71092CC052224332410
:101240001BAE1AAE12E0412E512C4C0E5D1EB3E0C7
:10125000AB2EA2E0BA2E01E0F1E06F2E712CA5C1F9
:101260002E313105C9F12F313105D4F42431310546
:1012700084F421313105A4F52430310569F125309C
:1012800031051CF437FF2AC025C02A30310511F57D
:1012900023C02631310554F12C313105D9F41CC05D
:1012A0002C3531058CF42A353105E4F42C33310525
:1012B0003CF426333105E4F42533310559F40CC0F0
:1012C0002035310539F40AC02C35310529F02F3588
:1012D000310554F010E00DC011E00BC012E009C060
:1012E00013E007C014E005C016E003C017E001C01A
:1012F00019E02531310509F494C026313105A4F5F2
:101300002430310509F467C025303105A4F42130BB
:10131000310509F465C02230310524F4232B09F48A
:101320005CC02EC12230310509F45DC02330310587
:1013300009F026C15BC02231310509F461C02331B7
:1013400031054CF42A30310509F443C0213131050F
:1013500009F016C14EC02331310509F458C02431BB
:10136000310509F00DC15AC02035310509F490C08E
:1013700021353105ACF42533310509F481C026331C
:1013800031054CF42C31310509F44EC02E313105B4
:1013900009F0F6C049C02C3331050CF0F1C073C020
:1013A0002C35310509F47EC02D3531054CF42A3534
:1013B000310509F471C02B35310509F0E1C06FC06A
:1013C0002D35310509F488C02E35310509F0D8C016
:1013D00086C0B2E07FC0E1E04EC01092CD05D2C021
:1013E0000093CD05CFC0B092CD05CCC0A092CD0565
:1013F000C9C01092E5050093E605B092E705C2C0AA
:10140000B092E5051092E6050093E705BBC0009396
:10141000E505B092E6051092E705B4C00093CF054C
:10142000B1C01092CF05AEC0C701B60120E030E0D8
:1014300040E251E40E94AE320E9488330E943D3067
:10144000F1E069317F0791F041E06A3174072CF4D3
:101450006851714009F094C00BC081E06C3278078C
:1014600049F06D52714009F08BC007C0A4E02FC055
:10147000B3E030C0E5E0EAAF85C0F6E0FAAF82C085
:1014800041E04BAF7FC0822F86538093E8057AC03E
:1014900054E05093CD0576C00093D00573C01092F0
:1014A000D00570C0C701B60120E030E040E251E451
:1014B0000E94AE320E9488330E943D3083E068393A
:1014C000780739F06959734009F05AC0A8E0AAAF0B
:1014D00059C0B7E0BAAF56C00093CE0553C01092C2
:1014E000CE0550C02630310534F42330310554F494
:1014F000772334F403C02E31310511F010E003C01E
:1015000015E001C018E02430310569F125303105BE
:1015100084F421303105B1F1223031051CF4232B44
:10152000C9F02EC022303105C1F02330310541F51C
:1015300017C028303105F1F02930310524F4253069
:101540003105F1F414C029303105B9F02E313105DF
:10155000B9F403C00093D10515C0B092D10512C0F3
:101560000093D2050FC0EFEFE093D2050BC01092AD
:10157000D20508C00093D30505C01092D30502C060
:10158000A092CC05112389F0930102C0220F331FD2
:101590001A95E2F7C90182219321892B21F0F5E008
:1015A000F093CC0502C0222A332A9981F401E90F75
:1015B000F11D10811123A9F0812F81548A3110F07F
:1015C00082E00DC09F5F9983C401BE016F5F7F4FB2
:1015D000A2010E94DE24892B09F000C681E08093DD
:1015E000CC058091CC05882309F0DFC519827724CA
:1015F0001CAE1DAE40E84EAF5FEB5FAF0F2EF0E0CC
:10160000AF2EF0E0BF2EF0E0CF2EF0E0DF2EF02D79
:10161000AEAABFAAC8AED9AE4424E6E06E2E73E0EF
:10162000572E0FC1EA80FB800C811D81C801B701D4
:1016300020E030E040E050E00E94CE2F181614F079
:101640006092CC058091CE05882381F08091CF05F2
:10165000882309F4F0C0C801B70123E333E34BEC5E
:1016600051E40E94AE327B018C01E5C08091CF0530
:10167000882351F0C801B70123E333E34BEC51E475
:101680000E94AE327B018C01E092D405F092D50528
:101690000093D6051093D705C8C02A813B814C81A1
:1016A0005D818091CF05882351F0CA01B90123E300
:1016B00033E34BEC51E40E94AE329B01AC01E12FCD
:1016C000FF27E7FDF095E954F040EE0FFF1FEE0F06
:1016D000FF1F61E070E06C0F7D1FE60FF71F218B8D
:1016E000328B438B548BA1C06A817B818C819D811D
:1016F0000E9488330E944230462E97C0AA80BB8049
:10170000CC80DD8092C08A819B81AC81BD818EAB13
:101710009FABA8AFB9AF8091CF05882309F485C0EE
:101720006EA97FA988AD99AD23E333E34BEC51E477
:101730000E94AE326EAB7FAB88AF99AF76C06A8144
:101740007B818C819D8120E030E040E050E00E9470
:10175000CE2F88230CF069C06092CC0566C0EA8069
:10176000FB800C811D81C801B70120E030E040E022
:1017700050E00E94CE2F882314F46092CC05C8015B
:10178000B7010E9488330E9442306093E4054DC047
:101790002A813B814C815D818091CF05882351F066
:1017A000CA01B90123E333E34BEC51E40E94AE32AA
:1017B0009B01AC012E833F834887598791E0792AAA
:1017C00034C02A813B814C815D818091CF05882383
:1017D00051F0CA01B90123E333E34BEC51E40E9419
:1017E000AE329B01AC012A873B874C875D87A2E024
:1017F0007A2A1BC02A813B814C815D818091CF0573
:10180000882351F0CA01B90123E333E34BEC51E4DF
:101810000E94AE329B01AC012E873F87488B598BCB
:10182000B4E07B2A02C05092CC058CAD9DADAEAD2C
:10183000BFAD7C018D01D801C701ECAE9DAFAEAF4D
:10184000BFAF9981F401E90FF11D10811123B9F0A7
:10185000812F81548A3110F082E00FC09F5F9983FD
:10186000C401BE016F5F7F4FAE014E5F5F4F0E94AC
:10187000DE24892B09F0C4C481E08093CC058091DB
:10188000CC05882309F091C48091BD05873041F0D3
:101890008091D2050E9461118091D3050E9484112C
:1018A00031FE13C08E01025E1F4F8091E805B80122
:1018B0000E94801C882309F477C4A9EEB5E0F801E2
:1018C0008CE001900D928150E1F7EAADE43009F42B
:1018D00063C1E53048F4E23051F1E33008F0B2C0C2
:1018E000E13009F0B1C10EC0FAADF63009F454C1CF
:1018F000F63008F4A7C0F73009F459C1F83009F000
:10190000A3C199C1C601B50120E030E040E050E03C
:101910000E94CE2F88230CF44CC18091BD058730E6
:1019200009F492C1C601B5010E941A048DC142E0BA
:10193000441619F054E1451649F4C601B5010E9458
:1019400088330E943D306730710520F083E080933A
:10195000CC0579C1772021F482E0481609F429C129
:10196000161617062CF44B0108948108910804C040
:101970008091E805882E9924582C8E01025E1F4F15
:10198000882DB8010E94801C882309F40DC438ED0D
:10199000A32E35E0B32E26E0C22ED12CCC0EDD1EB8
:1019A000780100E010E0672C7724C301002E02C00C
:1019B000959587950A94E2F780FF20C094E1491637
:1019C00099F4D5016D917D918D919C91F6012081C5
:1019D0003181428153810E94F42ED7016D937D9312
:1019E0008D939C9313970AC0F60180819181A28107
:1019F000B381F70180839183A283B3830F5F1F4F6D
:101A000044E050E0A40EB51EC40ED51EE40EF51E33
:101A10000330110551F68E01025E1F4F852DB8016E
:101A20000E94751C8091E80590E08815990509F0E1
:101A30000AC1A9EEB5E0F8018CE001900D92815049
:101A4000E1F701C1772009F478C08E010A5F1F4FCA
:101A500098EDE92E95E0F92ECC24DD24A72CBB24AB
:101A6000C5010C2C02C0959587950A94E2F780FF7A
:101A700035C08091D0058823F9F0D70151966D913A
:101A80007D918D919C9154975D962D913D914D91B5
:101A90005C9190970E94F52E9B01AC01F80160814A
:101AA0007181828193810E94F52ED8016D937D937F
:101AB0008D939C9313971CC0F80160817181828182
:101AC0009381D7012D913D914D915C910E94F52E0E
:101AD000F80160837183828393830AC0F701808158
:101AE0009181A281B381F80180839183A283B38322
:101AF0000894C11CD11C0C5F1F4F44E050E0E40E61
:101B0000F51E53E0C516D10409F0AACF6E817F817E
:101B1000888599852A853B854C855D85EE84FF8483
:101B200008891989A090D306B090D406C090D50634
:101B3000D090D60688240E946E04BE01665D7F4F59
:101B40008AAD853011F487E001C086E00E94801CD8
:101B5000882309F429C36AA57BA58CA59DA52EA57C
:101B60003FA548A959A9EAA8FBA80CA91DA9A090BE
:101B7000D306B090D406C090D506D090D60688245F
:101B80000E946E04A8EDB5E0FE01BA968CE00190CB
:101B90000D928150E1F757C09AAD963011F487E06D
:101BA00001C086E068ED75E00E94751C4DC077208D
:101BB00021F486E08093CC0547C008ED15E086E06F
:101BC000C82ED12CCC0EDD1EEE24FF24A72CBB2466
:101BD000C5010E2C02C0959587950A94E2F780FF07
:101BE0001CC0D8016D917D918D919C911397519658
:101BF0002D913D914D915C9154970E94F42EF601E8
:101C000020813181428153810E94F42ED8015D965A
:101C10006D937D938D939C9390970894E11CF11C98
:101C20000C5F1F4FE4E0F0E0CE0EDF1EF3E0EF1696
:101C3000F10471F608C08CE0E5EFF5E0DF011D92DC
:101C40008A95E9F701C0772422FC03C0772009F4C4
:101C500097C28091CE05882399F06CAD7DAD8EAD95
:101C60009FAD20E030E040E050E00E94CE2F88237E
:101C70003CF48091CD05843019F086E08093CC054A
:101C8000BBADBB2339F08091CD05823018F086E0E2
:101C90008093CC058091CC05882309F086C28E0103
:101CA0000A5F1F4FB8EDEB2EB5E0FB2ECC24DD24F0
:101CB000A72CBB24C5010C2C02C0959587950A94CE
:101CC000E2F780FF39C0EBADEE2309F03FC0809111
:101CD000D0058823F9F0D70151966D917D918D91B2
:101CE0009C9154975D962D913D914D915C9190976B
:101CF0000E94F52E9B01AC01F80160817181828107
:101D000093810E94F52ED8016D937D938D939C93C2
:101D100013971CC0F8016081718182819381D70182
:101D20002D913D914D915C910E94F52EF8016083BB
:101D30007183828393830AC0F70180819181A2819C
:101D4000B381F80180839183A283B3830894C11C7B
:101D5000D11C0C5F1F4F44E050E0E40EF51E53E031
:101D6000C516D10409F0A6CF8091CD05843048F482
:101D7000823008F04CC0882359F0813009F0F3C15B
:101D800020C0843009F0EFC1772009F4ECC18BC08A
:101D9000772009F488C06E817F81888599852A859E
:101DA0003B854C855D85EE84FF8408891989A09068
:101DB000D306B090D406C090D506D090D60688241D
:101DC00023C0772009F46FC06E817F818885998553
:101DD0002A853B854C855D85EE84FF8408891989B9
:101DE0008090CE05882061F4A091D405ACAFB0916D
:101DF000D505BDAFE091D605EEAFF091D705FFAFA9
:101E0000ACACBDACCEACDFAC0E946E04ACC181E02A
:101E100090E00090E70502C0880F991F0A94E2F74E
:101E20008095782209F43FC06EA97FA988AD99AD4D
:101E300020E030E040E050E00E94CE2F882309F0FF
:101E400043C0E091E505F0E0EE0FFF1FEE0FFF1F2E
:101E50008E010F5F1F4FE00FF11FC188D288E3880A
:101E6000F488C701B60120E030E040E050E00E9475
:101E7000CE2F8823E1F48091E60590E0880F991F2A
:101E8000880F991F080F191FD80151966D917D91E8
:101E90008D919C91549720E030E040E050E00E940A
:101EA000CE2F882321F486E08093CC055CC16EA9F7
:101EB0007FA988AD99AD20E030E040E050E00E947D
:101EC000CE2F882309F4F8C0E091E505F0E0EE0F8D
:101ED000FF1FEE0FFF1F8E010F5F1F4FD801AE0FC8
:101EE000BF1FE852FA4F15966D917D918D919C918F
:101EF000189720813181428153810E94F42E1B0169
:101F00002C01E091E605F0E0EE0FFF1FEE0FFF1F42
:101F10000E0F1F1FE852FA4FD80115966D917D9153
:101F20008D919C91189720813181428153810E942B
:101F3000F42E3B014C018CE0FE017296DF011D92F4
:101F40008A95E9F76EA97FA988AD99AD20E030E0C8
:101F500040E850E40E94AE322EA93FA948AD59ADE9
:101F60000E94AE327B018C01C201B101A20191013C
:101F70000E94AE329B01AC01C801B7010E94F42E51
:101F80007B018C01C401B301A40193010E94AE3214
:101F90009B01AC01C801B7010E94F42E7B018C01AA
:101FA00020E030E040E050E00E94CE2F882324F46F
:101FB00084E08093CC05F9C0C801B7010E943B338F
:101FC0007B018C01C201B101A40193010E94E9319E
:101FD0009B01AC0117FB109517F91095C801B701CB
:101FE0000E94D52F6B017C018091CD05833021F4B7
:101FF000F7FAF094F7F8F0946EA97FA988AD99AD3F
:1020000020E030E040E050E00E94CE2F88236CF4C6
:10201000F7FAF094F7F8F0944EA95FA968AD79AD9E
:1020200070584EAB5FAB68AF79AF0091E505A02E5D
:10203000BB24AA0CBB1CAA0CBB1C8E010F5F1F4F3C
:10204000A00EB11EC401B301A70196010E94AE32D9
:102050009B01AC01C201B1010E94F42E20E030E0EE
:1020600040E05FE30E94AE32D50151966D937D93BF
:102070008D939C9354978091E60590E0880F991F6B
:10208000880F991F080F191FC201B101A7019601FE
:102090000E94AE329B01AC01C401B3010E94F52E37
:1020A00020E030E040E05FE30E94AE32F801618B57
:1020B000728B838B948B15C0E091E605F0E0EE0FF8
:1020C000FF1FEE0FFF1FEC0FFD1F2289338944898C
:1020D0005589C701B6010E94E9316EAB7FAB88AF6D
:1020E00099AF9091CD052091E5050091E605E0902E
:1020F000E7058090CE05882061F4F091D405FCAF0F
:102100004091D5054DAF5091D6055EAF6091D70592
:102110006FAF00D000D00F92EDB7FEB731964EA949
:102120005FA968AD79ADADB7BEB711964D935D931C
:102130006D937C93149780E0923009F481E084835E
:1021400088ED95E0BE016A5F7F4FAE014E5E5F4F46
:10215000ACACBDACCEACDFAC0E9460050F900F9074
:102160000F900F900F908091CC058823F1F4A8ED8B
:10217000B5E0FE0136968CE001900D928150E1F7BA
:102180008091D105882369F00E94AD241092CB057F
:102190008091D105823019F40E94000402C010928F
:1021A000D1058091CC0501C08AE0EF960FB6F89476
:1021B000DEBF0FBECDBFCF91DF911F910F91FF907A
:1021C000EF90DF90CF90BF90AF909F908F907F90D7
:1021D0006F905F904F903F902F900895CA80DB8062
:1021E000EC80FD80C701B6010E9488330E943D301B
:1021F0009B01173409F434C81D3409F0D6C972C9DB
:102200001F3484F41D340CF010CB1C340CF06CCA59
:1022100019340CF042CA163409F404CA173409F010
:1022200002CB03CB143509F49ACA153554F4123590
:1022300009F469CA13350CF082CA103509F0F3CAE3
:102240005DCA193509F4BDCA1A3509F4D3CA18355F
:1022500009F0E9CA9DCAECECF5E085E3DF011D92C7
:102260008A95E9F78091CF069091D006A091D1068A
:10227000B091D2068093D4059093D505A093D6054E
:10228000B093D7051092E50591E09093E60582E0C2
:102290008093E7059093D0058091E805BF01635EC8
:1022A0007F4F0E94801C882319F48AE00E947A2ABA
:1022B000089510920001249A259A2C9808952C983C
:1022C00008951F93182F282F332727FD30958091CD
:1022D000000190E02817390771F00E94AD24112306
:1022E00039F0111614F42D9801C02D9A2C9A01C0C2
:1022F0002C98109300011F910895109201013B9AB0
:1023000043980895439808951F93182F80910101D1
:10231000181749F00E94AD24113011F4439A01C0FE
:102320004398109301011F910895E0ECF0E0808143
:102330008D7F80831092C50087E68093C400E1EC16
:10234000F0E08081806180838081886080838081EB
:10235000806880830895282FE09104019E2F9F5F5D
:10236000903431F490E004C08091BE0584FD0FC02C
:10237000809105019817C1F3F0E0EF57F94F2083E2
:10238000909304018091C10080628093C100089500
:102390001F920F920FB60F9211248F939F93EF937A
:1023A000FF9380910501E82FF0E0EF57F94F9081FE
:1023B0009093C600982F9F5F903409F490E090931B
:1023C000050180910401981729F48091C1008F7D47
:1023D0008093C100FF91EF919F918F910F900FBE5D
:1023E0000F901F9018959091030180910201891719
:1023F00011F48FEF0895E92FF0E0EF5FF94F80813E
:10240000E92FEF5FE03809F4E0E0E093030108957D
:10241000809102018093030108951F920F920FB6DD
:102420000F9211242F933F934F935F936F937F935A
:102430008F939F93AF93BF93EF93FF932091C60029
:102440002132A1F0223218F42831B9F413C02F330D
:1024500019F02E3791F404C08091BE05816003C04D
:102460008091BE0582608093BE0518C08091BE0534
:102470008860F9CF0E94000411C0E09102019E2FF4
:102480009F5F903809F490E080910301981731F034
:10249000F0E0EF5FF94F208390930201FF91EF91FD
:1024A000BF91AF919F918F917F916F915F914F916C
:1024B0003F912F910F900FBE0F901F9018951F9274
:1024C0000F920FB60F9211242F933F934F935F9368
:1024D0006F937F938F939F93AF93BF93EF93FF93EC
:1024E00086B190E08095909587709070892B91F0DF
:1024F000309903C00E9400040DC0319904C080913E
:10250000BE05886005C0329905C08091BE05826015
:102510008093BE05FF91EF91BF91AF919F918F91F5
:102520007F916F915F914F913F912F910F900FBECF
:102530000F901F901895CF93DF938091BE0588234D
:1025400009F457C08091BE05C82FD0E0CE01807637
:102550009070892BE9F086E08093BD05C6FF10C01E
:102560008FEF0E94D92E81E00E94502A8091BE05F3
:102570008F7E8093BE058091BE0584FFFCCF03C093
:102580008EEF0E94D92E8091BE058F798093BE0573
:10259000C4FF04C081E08093BC052BC0C0FF07C00E
:1025A0000E94D52A8091BE058E7F8093BE05C3FF11
:1025B00007C00E9479158091BE05877F8093BE0574
:1025C000C2FF07C00E9483158091BE058B7F809358
:1025D000BE05C1FF0EC00E946F158091E40681FF09
:1025E00003C081E08093CB058091BE058D7F8093F1
:1025F000BE05DF91CF91089580E066E071E00E9412
:10260000EC1C882369F080910601882361F086E044
:1026100091E00E94392A86E091E00E94EC0801C016
:102620008AE00E947A2A81E066E071E00E94EC1C58
:10263000882321F48AE00E947A2A08958091060175
:10264000882351F086E091E00E94392A86E091E0EB
:102650000E94EC080E947A2A0895DF92EF92FF927E
:102660000F931F93DF93CF93CDB7DEB729970FB6A4
:10267000F894DEBF0FBECDBF7C01FC0180818432A7
:1026800009F009C181E089838181873481F188342F
:1026900074F48432C1F0853234F4882389F08332B3
:1026A00009F097C01AC0833409F093C02AC08E3451
:1026B00009F469C08835F1F1883409F08AC04CC04A
:1026C0000E94462AF3C082E08983F7018281882331
:1026D00009F0E6C00E947B2DE9C082E08983F70102
:1026E0008281882309F0DCC00E94BD2CDFC082E01B
:1026F0008983F7018281882309F0D2C00E94D22BFE
:10270000D5C082E08983F7018281882309F0C8C09F
:102710008091BD05873021F40E94000485E007C048
:10272000882309F0BFC087E08093BD0584E00E9444
:10273000502ABCC082E08983F7018281882309F096
:10274000AFC08091BD05863009F0B0C083E00E9423
:10275000502A1092BD05AAC08091E40684FD02C0F3
:1027600017E0A5C08091BD05882319F0863009F0D7
:1027700099C00E94BE048091BC05882309F096C0D0
:102780000E94FC1293C082E08983F7018281882332
:1027900019F0DD24D3941EC080E0B7010E94EC1C28
:1027A000882329F080E0B7010E94982C03C08AE0BA
:1027B0000E947A2A81E0B7010E94EC1C882321F450
:1027C0008AE00E947A2A72C081E0B7010E94982CA8
:1027D0006DC0DD24C7018E010F5F1F4FB801AE0130
:1027E0004E5F5F4F0E94DE24892B09F45DC0998102
:1027F000F701E90FF11D80818D3309F051C0892F58
:102800008F5F8983DD2041F1482F50E02981822F9D
:1028100090E0FC01E41BF50BEE0DFF1DD701A80FA6
:10282000B91F8C9180838C912F5F2983882371F746
:10283000C7010E94EC08182F8823C9F56A817B81A3
:102840008C819D810E9488330E944230DC01CB0143
:10285000B7010E94E11C2BC0C701B801AE014A5F5D
:102860005F4F0E94DE24892BF9F08981E80EF11C6C
:10287000F70180818823A1F46A817B818C819D810D
:102880000E943D30DC01CB014E815F8168857985F6
:102890000E94781A03C0C7010E94EC08182F07C0D5
:1028A00013E005C01BE003C011E001C010E0812F60
:1028B00029960FB6F894DEBF0FBECDBFCF91DF9142
:1028C0001F910F91FF90EF90DF9008951F9311E0FB
:1028D00046C02A3011F02D30B1F40E949B12809135
:1028E000BC05882309F041C0E0914C01EE2349F07A
:1028F000F0E0EA5FFE4F108286E091E00E942D1327
:1029000017C080E015C080914D01882319F029324D
:1029100031F512C0213218F12F3209F1283219F4A1
:1029200010934D011CC090914C01953440F08DE006
:102930000E947A2A10924C0110924D0110C0822FF1
:102940008156E92FF0E09F5F8A3120F4EA5FFE4F65
:10295000205202C0EA5FFE4F208390934C010E94F8
:10296000F311282F8F3F09F0B4CF1F9108951092D3
:102970004C0110924D010E944B2A87B1887F87B984
:1029800088B1876088B9ECE6F0E080818760808359
:10299000E8E6F0E080818260808308958091E4061B
:1029A00082FF02C0289A01C028988091BD0583301B
:1029B000C1F48091D706809375018091CE0690E096
:1029C000A0E0B0E00297A109B109880F991FAA1FE2
:1029D000BB1F81958093740180916F00826080930A
:1029E0006F0008951F920F920FB60F9211248F93CC
:1029F0009F939BB18091D7068C71937E892B8BB965
:102A00001092B1009F918F910F900FBE0F901F9069
:102A100018959B01AC01203283E0380780E048071D
:102A200080E0580720F420E233E040E050E060E02E
:102A300070E788E399E30E94C633C901DA01803068
:102A400020E0920721E0A20720E0B20730F4BC01A9
:102A50009C0140E050E091E02FC0803020E09207E0
:102A600028E0A20720E0B207A0F423E0B695A795DE
:102A7000979587952A95D1F7BC019C0140E050E0DD
:102A8000A3E0220F331F441F551FAA95D1F792E0F0
:102A900013C0F6E0B695A79597958795FA95D1F767
:102AA000BC019C0140E050E0E6E0220F331F441FD0
:102AB000551FEA95D1F793E080918100887F982B8C
:102AC0009093810070938900609388002093620145
:102AD00030936301409364015093650108958091A0
:102AE000BD05823029F483E08093BD050E94CE1499
:102AF00008958091BD05833029F484E08093BD055D
:102B00001092CB050895E0917201F0917301309716
:102B1000C1F1658576858785908920915E01309128
:102B20005F014091600150916101621B730B840B46
:102B3000950B0E94722010926A0110926B01109204
:102B40006C0110926D0160E070E080E090E00E9406
:102B5000091580E091E7A2E0B0E0809366019093D0
:102B60006701A0936801B093690110925E01109211
:102B70005F01109260011092610182E08093BD05B7
:102B800008951092BD05089584E2EEE4F1E0DF01BE
:102B90001D928A95E9F760E273E080E090E00E9480
:102BA0000915109273011092720110927601089526
:102BB00080916F008D7F80936F009091F4069F3F0E
:102BC00021F48091BE0585FF0BC0892F90E00E9403
:102BD00099258091E40682FF02C028980895289ADA
:102BE00008958AB18C6F8AB98BB183709091D706A2
:102BF000892B8BB9209AE1E8F0E080818F7E808379
:102C0000808188608083E0E8F0E080818D7F808330
:102C100080818E7F808380818F73808380818F7C91
:102C200080831092B0001092B100E0E7F0E0808164
:102C3000816080830E94CE140E94D81508951F924F
:102C40000F920FB60F921124EF92FF920F931F93E2
:102C50002F933F934F935F936F937F938F939F93A4
:102C6000AF93BF93CF93DF93EF93FF938091760160
:102C7000882309F06EC39BB120917501822F807E5D
:102C80009F71892B8BB98BB1837E822B8BB98091FD
:102C900074018093B20082E08093B10081E0809360
:102CA000760178948091720190917301892B09F0DB
:102CB0007FC00E941E1DEC019093730180937201EE
:102CC000009709F46EC08091BD058330D1F46BA1EB
:102CD0007CA18DA19EA160936A0170936B0180938A
:102CE0006C0190936D010E94091580E091E7A2E0CC
:102CF000B0E08093660190936701A0936801B09360
:102D000069012BA53CA54DA55EA5DA01C901B595C4
:102D1000A79597958795820F931FA41FB51F809342
:102D20006E0190936F01A0937001B09371012D8596
:102D30003E854F855889DA01C901B595A7959795C4
:102D40008795B095A095909581959F4FAF4FBF4FB8
:102D500080934E0190934F01A0935001B093510185
:102D60008093520190935301A0935401B093550165
:102D70008093560190935701A0935801B093590145
:102D800020935A0130935B0140935C0150935D01A5
:102D900010925E0110925F01109260011092610129
:102DA00007C00E94D8158091BE0584608093BE053F
:102DB000E0917201F0917301309709F4C1C2208152
:102DC0002093750140914E0150914F016091500147
:102DD0007091510181819281A381B481480F591F63
:102DE0006A1F7B1F40934E0150934F016093500127
:102DF000709351011416150616061706C4F52460C3
:102E00002093750180915A0190915B01A0915C0122
:102E1000B0915D01481B590B6A0B7B0B40934E012F
:102E200050934F01609350017093510125FF0CC0E6
:102E30008091BF059091C005A091C105B091C205D8
:102E40000197A109B1090BC08091BF059091C00500
:102E5000A091C105B091C2050196A11DB11D80933D
:102E6000BF059093C005A093C105B093C2054091E2
:102E70005201509153016091540170915501858127
:102E80009681A781B085480F591F6A1F7B1F409309
:102E900052015093530160935401709355011416DD
:102EA000150616061706D4F52091750128602093A3
:102EB000750180915A0190915B01A0915C01B091E4
:102EC0005D01481B590B6A0B7B0B409352015093D9
:102ED0005301609354017093550126FF0CC08091FB
:102EE000C3059091C405A091C505B091C605019791
:102EF000A109B1090BC08091C3059091C405A091AF
:102F0000C505B091C6050196A11DB11D8093C305ED
:102F10009093C405A093C505B093C6054091560192
:102F200050915701609158017091590181859285A6
:102F3000A385B485480F591F6A1F7B1F4093560114
:102F40005093570160935801709359011416150658
:102F500016061706D4F5209175012061209375019E
:102F600080915A0190915B01A0915C01B0915D014B
:102F7000481B590B6A0B7B0B40935601509357012A
:102F8000609358017093590127FF0CC08091C705C9
:102F90009091C805A091C905B091CA050197A109F2
:102FA000B1090BC08091C7059091C805A091C905D2
:102FB000B091CA050196A11DB11D8093C7059093DC
:102FC000C805A093C905B093CA0520915E01309150
:102FD0005F0140916001509161012F5F3F4F4F4F62
:102FE0005F4F20935E0130935F01409360015093E7
:102FF000610185859685A785B089281739074A0715
:103000005B0708F097C18091BD05843009F05BC073
:1030100020916201309163014091640150916501FA
:103020008091660190916701A0916801B09169015A
:10303000280F391F4A1F5B1F2093660130936701D9
:103040004093680150936901213002EE300704E09B
:10305000400700E0500708F473C12050324E44404E
:10306000504020936601309367014093680150936C
:10307000690120916A0130916B0140916C0150917E
:103080006D0163A574A585A596A5621773078407CE
:10309000950740F00E94D8158091BE05846080930A
:1030A000BE054EC179018A01E61AF70A080B190B11
:1030B000C801B701E0926A01F0926B0100936C01C4
:1030C00010936D016CC087A590A9A1A9B2A928177A
:1030D00039074A075B0708F065C02091620130910B
:1030E0006301409164015091650180916601909166
:1030F0006701A0916801B0916901280F391F4A1F2B
:103100005B1F2093660130936701409368015093E1
:103110006901213002EE300704E0400700E050076B
:1031200008F40EC12050324E4440504020936601B6
:1031300030936701409368015093690183A594A57A
:10314000A5A5B6A520916A0130916B0140916C0153
:1031500050916D01820F931FA41FB51F80936A01C8
:1031600090936B01A0936C01B0936D0127A930ADD2
:1031700041AD52AD82179307A407B50740F02093E5
:103180006A0130936B0140936C0150936D01609123
:103190006A0170916B0180916C0190916D010E94A8
:1031A0000915CEC083A994A9A5A9B6A928173907DE
:1031B0004A075B0708F4A2C0281739074A075B07CC
:1031C00079F520916A0130916B0140916C01509129
:1031D0006D0187A990ADA1ADB2AD281739074A0797
:1031E0005B0729F480E091E7A2E0B0E010C080E046
:1031F00092EEA4E0B0E02091660130916701409129
:10320000680150916901821B930BA40BB50B80934D
:10321000660190936701A0936801B093690190C023
:1032200020916201309163014091640150916501E8
:103230008091660190916701A0916801B091690148
:10324000280F391F4A1F5B1F2093660130936701C7
:103250004093680150936901213012EE310714E068
:10326000410710E0510708F46BC02050324E444033
:10327000504020936601309367014093680150935A
:10328000690120916A0130916B0140916C0150916C
:103290006D0180916E0190916F01A0917001B091CC
:1032A000710182179307A407B50748F483A594A575
:1032B000A5A5B6A5281B390B4A0B5B0B04C0569578
:1032C00047953795279520936A0130936B0140937A
:1032D0006C0150936D0127A130A541A552A58091A5
:1032E0006A0190916B01A0916C01B0916D01821700
:1032F0009307A407B50708F04ACF41CF27A930ADFF
:1033000041AD52AD80916A0190916B01A0916C0129
:10331000B0916D0182179307A407B50789F0209338
:103320006A0130936B0140936C0150936D01CA01A7
:10333000B90135CF10927301109272010E940F1DD6
:10334000809175019091D70689278093750110921D
:103350007601FF91EF91DF91CF91BF91AF919F9156
:103360008F917F916F915F914F913F912F911F911D
:103370000F91FF90EF900F900FBE0F901F90189538
:10338000F999FECF92BD81BD81E08FBB80B50895D4
:10339000F894F999FECF92BD81BD81E08FBB40B515
:1033A0004627842F992787FD9095262F30E082238A
:1033B0009323892B39F06F3F19F060BD84E006C07C
:1033C00084E104C0442321F060BD84E28FBBF99AFC
:1033D000789408958F929F92AF92BF92CF92DF928E
:1033E000EF92FF920F93DF93CF9300D0CDB7DEB76C
:1033F0005C016B017A014A0100E01EC0002319F054
:1034000021E030E008C0202F332727FD3095222708
:10341000330F221F3327F60161916F01062F020F30
:103420009C012F5F3F4F3A8329830E94C81908945B
:103430008108910889819A8181149104F9F6C70164
:103440008A0D9B1D602F0E94C8190F900F90CF917D
:10345000DF910F91FF90EF90DF90CF90BF90AF90F2
:103460009F908F900895CF93DF93EC01FB019A0119
:1034700090E0B1E019C0F999FECFF2BDE1BDBFBB4C
:10348000A0B5992319F081E090E008C0892F992711
:1034900087FD90958827990F881F992731969A2F35
:1034A000980FA993215030402115310521F7460F7F
:1034B000571FF999FECF52BD41BD81E08FBB80B54A
:1034C00020E030E0981711F421E030E0C901DF91ED
:1034D000CF91089580E090E065E00E94C81981E0F6
:1034E00090E061EC76E046E350E00E94EA1908952E
:1034F000EF92FF920F931F93CF93DF93EC017A012A
:103500008B01FC018731910540F4EC5CFF4FEE0F1D
:10351000FF1F0590F491E02D099486E01FC1CB01B7
:10352000BA0120E030E040E050E00E94CE2F1816B3
:1035300014F088E013C1CC0FDD1FCC0FDD1FCF537B
:10354000D94FE882F9820A831B8305C1CB01BA01F6
:1035500020E030E040E450E40E94CE2F882314F4B1
:1035600089E0FCC0C801B7010E9411330E944230BB
:103570006093CE06F0C04093CF065093D006609380
:10358000D1067093D206E7C04093D3065093D40679
:103590006093D5067093D606DEC0CB01BA010E94B7
:1035A00088330E9442306093D706D5C0CB01BA0160
:1035B0000E9411330E9442306093F406CCC0CB01CC
:1035C000BA0120E030E040E752E40E94AE3220E051
:1035D00030E040E752E40E94AE326093DC06709324
:1035E000DD068093DE069093DF06B5C0DB01CA01DD
:1035F000BF778093E0069093E106A093E206B09334
:10360000E306A9C04093D8065093D9066093DA0622
:103610007093DB06A0C0CB01BA010E9411330E9457
:1036200042306093F60697C0CB01BA010E94113375
:103630000E9442306093F5068EC0CB01BA0120E0B3
:1036400030E040E050E00E94CE2F882321F08091AE
:10365000E406816011C08091E4068E7F0DC0CB012D
:10366000BA0120E030E040E050E00E94CE2F8823F5
:1036700031F08091E40682608093E4066CC0809112
:10368000E4068D7FF9CFCB01BA0120E030E040E0C5
:1036900050E00E94CE2F882321F08091E4068460C0
:1036A000EBCF8091E4068B7FE7CFCB01BA0120E01E
:1036B00030E040E050E00E94CE2F882321F080913E
:1036C000E406886003C08091E406877F8093E40667
:1036D0000E94202640C0CB01BA0120E030E040E04B
:1036E00050E00E94CE2F882321F08091E406806173
:1036F000C3CF8091E4068F7EBFCFCB01BA010E9479
:1037000088330E9442306093E50625C04093E60668
:103710005093E7066093E8067093E9061CC0409357
:10372000EA065093EB066093EC067093ED0613C027
:10373000CB01BA010E9411330E9442307093EF0610
:103740006093EE0608C04093F0065093F106609334
:10375000F2067093F3060E946A1A80E0DF91CF911F
:103760001F910F91FF90EF900895882309F45AC09C
:1037700080E090E0AAE7B3E48093C1069093C2068C
:10378000A093C306B093C4068093C5069093C60663
:10379000A093C706B093C8068093C9069093CA0643
:1037A000A093CB06B093CC062AE02093CE0680935C
:1037B000CF069093D006A093D106B093D20680E0B6
:1037C00090E0AAEFB3E48093D3069093D406A0933D
:1037D000D506B093D60680E090EAACE0B7E48093DB
:1037E000DC069093DD06A093DE06B093DF068DEC39
:1037F0009CECACECBDE38093D8069093D906A093E3
:10380000DA06B093DB0680EC8093D7068DEC9CEC57
:10381000ACE4BDE38093E0069093E106A093E2065A
:10382000B093E30682E08093E4061092E50680E020
:1038300090E0A8ECB1E48093E6069093E706A093AD
:10384000E806B093E90680E090E0AAE7B3E480934D
:10385000EA069093EB06A093EC06B093ED0684E69F
:1038600090E09093EF068093EE0680E090E0A0E871
:10387000BFE38093F0069093F106A093F206B09315
:10388000F30699E19093F40683E08093F506909314
:10389000F6060E946A1A089580E090E00E94C0191E
:1038A000853079F481EC96E061E070E046E350E029
:1038B0000E94331A20E0892B09F421E081E02827B7
:1038C00012C0853078F481EC96E061E070E043E26C
:1038D00050E00E94331A892B29F080E00E94B51B2A
:1038E00021E001C020E0822F08959DE0899FC00162
:1038F000112480509E4F4CE050E00E94EA19089538
:103900000F931F93CF93DF93162F072F9DE0899F6F
:10391000E0011124C050DE4F862F972FBE014CE0EE
:1039200050E00E94331A892B11F081E00FC0E12F83
:10393000F02F8CE0DF011D928A95E9F7CE01612F0F
:10394000702F4CE050E00E94EA1980E0DF91CF91A7
:103950001F910F910895EF92FF921F93DF93CF93E2
:10396000CDB7DEB72C970FB6F894DEBF0FBECDBF34
:103970000E944C1C882341F48AE00E947A2A81E04C
:103980000E94B51B0E947B2D10E07E010894E11C73
:10399000F11C812FB7010E94801C882319F48AE052
:1039A0000E947A2A1F5F1830A1F72C960FB6F89460
:1039B000DEBF0FBECDBFCF91DF911F91FF90EF9083
:1039C000089597E4899FC001112480509D4F46E4DB
:1039D00050E00E94EA1908950F931F93CF93DF934D
:1039E0008B0197E4899FE0011124C050DD4FCB018A
:1039F000BE0146E450E00E94331A892B11F081E0A9
:103A000009C0F8011082CE01B80146E450E00E94DE
:103A1000EA1980E0DF91CF911F910F910895909165
:103A20009D0580919E05981741F080919E058F5FBE
:103A3000823109F480E080939E05089590919D0560
:103A400080919E05981719F420E030E008C090910D
:103A50009E058BE3989F9001112429583E4FC90180
:103A6000089590919E0520E080919F05981709F494
:103A700021E0822F0895EF92FF920F931F9360939E
:103A8000A0057093A1058093A2059093A3052093B0
:103A9000A4053093A5054093A6055093A705E09291
:103AA000A805F092A9050093AA051093AB051F91F4
:103AB0000F91FF90EF9008958F929F92AF92BF92D7
:103AC000CF92DF92EF92FF920F931F93CF93DF93EA
:103AD000EC016B01009709F460C08AA1882309F00A
:103AE0005CC0ED88FE880F89188DFB01B588A6881B
:103AF0009788808CC801B7012B2D3A2D492D582D60
:103B00000E94CE2F88230CF048C0C801B701A8013D
:103B100097010E94AE327B018C016091DC067091AE
:103B2000DD068091DE069091DF06905820E030E0BF
:103B300040E050EC0E94AE322D8D3E8D4F8D58A14D
:103B40000E94AE329B01AC01C801B7010E94F52E64
:103B50000E943B337B018C016B2D7A2D892D982D92
:103B60009701A8010E94CE2F882324F4EB2CFA2C75
:103B7000092D182D6B2D7A2D892D982D9701A801CF
:103B80000E94CE2F882349F0C701D801F601858B0A
:103B9000968BA78BB08F81E081A3DF91CF911F918E
:103BA0000F91FF90EF90DF90CF90BF90AF909F90DC
:103BB0008F9008952F923F924F925F926F927F92D3
:103BC0008F929F92AF92BF92CF92DF92EF92FF922D
:103BD0000F931F93DF93CF93CDB7DEB768970FB6E0
:103BE000F894DEBF0FBECDBF1C016A017B01280126
:103BF0003901DC01D7966D917D918D919C91DA9779
:103C00000E946E304B015C01A70196010E94AE320A
:103C10000E94BB2F0E9442307B018C01F10163A303
:103C200074A385A396A3C501B401A30192010E94C8
:103C3000AE320E94BB2F0E94423069877A878B8701
:103C40009C87D10197966D937D938D939C939A97C2
:103C50009B966D917D918D919C919E9722E330E092
:103C600040E050E00E94A7330E94703020E030E036
:103C700040E752E40E94AE320E943D302B013C01ED
:103C8000C801B7010E946E307B018C01C301B201F3
:103C90000E9470306D837E838F839887C501B40145
:103CA000A50194010E94AE325B016C01C801B7010D
:103CB000A80197010E94AE326D877E878F87988B0F
:103CC0006D817E818F8198859B01AC010E94F52ECC
:103CD000698B7A8B8B8B9C8BC601B5012D853E85BC
:103CE0004F8558890E94F42E29893A894B895C892D
:103CF0000E94D52F0E94BB2F0E943D3069837A839A
:103D00008B839C8369857A858B859C850E946E3028
:103D10009B01AC010E94AE326D8B7E8B8F8B988F96
:103D2000A60195010E94F42E7B018C017094609491
:103D300050944094411C511C611C711CC301B20180
:103D40000E9470309B01AC010E94F52E9B01AC01DA
:103D5000C801B7010E94D52F0E94AB30F101A584A4
:103D6000B684C784D0888601750129813A814B8148
:103D70005C81E21AF30A040B150B0E943D30A80186
:103D80009701261B370B480B590BDA01C90157FF66
:103D90004AC0C601B5010E9470309B01AC0169891F
:103DA0007A898B899C890E94AE322D853E854F850C
:103DB00058890E94F42E2D893E894F89588D0E9482
:103DC000F52E7B018C016D817E818F81988520E0AD
:103DD00030E040E850E40E94AE329B01AC01C801E3
:103DE000B7010E94D52F0E94BB2F0E943D30AC012D
:103DF000CB01DA01BC01CD0197FF04C060E070E0A7
:103E000080E090E069837A838B839C83A616B70653
:103E1000C806D90624F4A982BA82CB82DC8280E06B
:103E200090E0A0E0B0E029813A814B815C81F10112
:103E300027A730AB41AB52AB820F931FA41FB51F16
:103E400083AB94ABA5ABB6AB68960FB6F894DEBF68
:103E50000FBECDBFCF91DF911F910F91FF90EF90DB
:103E6000DF90CF90BF90AF909F908F907F906F909A
:103E70005F904F903F902F9008952F923F924F92D6
:103E80005F927F928F929F92AF92BF92CF92DF927A
:103E9000EF92FF920F931F93CF93DF93D0909D05E6
:103EA0008091DC069091DD06A091DE06B091DF06E0
:103EB0001C012D0157FA509457F8509400E010E07F
:103EC000C0E0D0E0BB24B3943BE3C32E72C0DD203E
:103ED00011F422E1D22EDA94209709F463C001157F
:103EE000110509F45FC0A98C9A8C8B8C7C8C6D8930
:103EF0007E898F89988D2A2D392D482D572D0E9426
:103F0000CE2F882309F44EC08AA1882309F041C02E
:103F1000F801E588F6880789108D6A2D792D882D9E
:103F2000972DA80197010E94DC31181694F5C8015D
:103F3000B701A80197010E94AE327B018C01C2013A
:103F4000B10120E030E040E050EC0E94AE322D8D17
:103F50003E8D4F8D58A10E94AE329B01AC01C8012D
:103F6000B7010E94F52E0E943B33162F072FF82E23
:103F7000E92E6A2D792D882D972D212F302F4F2D49
:103F80005E2D0E94CE2F87FD04C0A12E902E8F2C77
:103F90007E2C8A2D992DA82DB72D8D8B9E8BAF8BC6
:103FA000B88FB9A2DC9CC00111248E01EC01C95864
:103FB000DE4F80919E05D81609F089CFF0909E05BE
:103FC00020E030E000E010E09BE3E92E11C0FE9C11
:103FD000E0011124C958DE4FC901B801AE010E94A9
:103FE0005C1DF394F2E1FF1609F4FF2498018E01A1
:103FF00080919D05F81659F7C901B80140E050E0DD
:104000000E945C1D70909E05C0E0D0E08BE3582EAE
:1040100035C0759C4001112487E791E0880E991EF8
:10402000209731F189A1882321F4F40181A188230B
:10403000F9F0E988FA880B891C896D897E898F8956
:10404000988DA80197010E94D52F5B016C01F401A6
:10405000658976898789908DA80197010E94D52F5F
:104060008B019C01CE01B601A5010E94DA1D19A2A7
:104070007394F2E17F1609F47724E40180919D05A1
:10408000781639F6E988FA880B891C896D897E894A
:104090008F89988DA80197010E94D52F5B016C0133
:1040A00060E070E080E090E0A80197010E94D52FC9
:1040B0008B019C01CE01B601A5010E94DA1D19A257
:1040C000DF91CF911F910F91FF90EF90DF90CF90F4
:1040D000BF90AF909F908F907F905F904F903F9058
:1040E0002F900895AF92BF92CF92DF92EF92FF92FE
:1040F0000F931F93CF93DF935B016C0190919E050B
:104100008BE3989FE0011124C958DE4FC601B50129
:104110000E9470302D8D3E8D4F8D58A10E94AE3281
:104120007B018C016D857E858F8598890E9470301A
:104130009B01AC01C801B7010E94D52F6D8F7E8F06
:104140008F8F98A3AD86BE86CF86D88A80E090E018
:10415000A0E0B0E08D8B9E8BAF8BB88F898F9A8F4C
:10416000AB8FBC8F1AA281E089A30E943D1FDF9113
:10417000CF911F910F91FF90EF90DF90CF90BF9064
:10418000AF9008952F923F924F925F926F927F92DD
:104190008F929F92AF92BF92CF92DF92EF92FF9257
:1041A0000F931F93DF93CF93CDB7DEB7C355D040A6
:1041B0000FB6F894DEBF0FBECDBF29013A0123969A
:1041C000ACAEBDAECEAEDFAE239724968FAE2497B5
:1041D00030919D052BE3329FA001112449585E4F79
:1041E0005A8F498F2091C1063091C2064091C30673
:1041F0005091C4062BAF3CAF4DAF5EAF0E94AE32C4
:104200000E947E3229966FAF29972A967FAF2A9710
:104210002B968FAF2B972C969FAF2C978091C5062E
:104220009091C606A091C706B091C8068FAB98AF13
:10423000A9AFBAAFC301B2012FA938AD49AD5AAD8C
:104240000E94AE320E947E322D966FAF2D972E9631
:104250007FAF2E972F968FAF2F9760969FAF609767
:104260002091C9063091CA064091CB065091CC06E8
:104270002BAB3CAB4DAB5EABC801B7010E94AE327D
:104280000E947E3261966FAF619762967FAF6297B0
:1042900063968FAF639764969FAF6497A98DBA8D2D
:1042A0001C922091A0053091A1054091A20550914A
:1042B000A3052C968CAD9DADAEADBFAD2C978217EE
:1042C0009307A407B50724F480E2A98DBA8D8C93D7
:1042D0004090A4055090A5056090A6057090A70594
:1042E00060968CAD9DADAEADBFAD60978415950564
:1042F000A605B7052CF4A98DBA8D8C9180648C939A
:10430000E090A805F090A9050091AA051091AB05D1
:1043100064968CAD9DADAEADBFAD64978E159F0517
:10432000A007B1072CF4A98DBA8D8C9180688C936D
:104330002C96ACACBDACCEACDFAC2C97A21AB30AB9
:10434000C40AD50AE98DFA8DA182B282C382D482D1
:10435000D7FE0BC088279927DC018A199B09AC0975
:10436000BD0981839283A383B48360962CAD3DAD58
:104370004EAD5FAD609724193509460957093901DB
:104380004A01A98DBA8D15962D933D934D935C935B
:10439000189757FF0DC088279927DC01821B930BC4
:1043A000A40BB50BE98DFA8D85839683A783B0871F
:1043B00064962CAC3DAC4EAC5FAC64972E183F08B5
:1043C000400A510AA201910157FE07C02227332754
:1043D000A9012219330944095509A98DBA8D1996E5
:1043E0002D933D934D935C931C971596ED90FD9006
:1043F0000D911C911897FD0181819281A381B48157
:104400008E159F05A007B10710F4D801C7018217C8
:104410009307A407B50710F4DA01C901E98DFA8DF5
:1044200085879687A787B08B0097A105B10509F40A
:104430007AC2C601B5010E9470302BAD3CAD4DADC6
:104440005EAD0E94D52F6FA778AB89AB9AABC40144
:10445000B3010E9470302FA938AD49AD5AAD0E940A
:10446000D52F6BA77CA78DA79EA7C201B1010E9483
:1044700070302BA93CA94DA95EA90E94D52F6FA32E
:1044800078A789A79AA76FA578A989A99AA99B0156
:10449000AC010E94AE327B018C016BA57CA58DA581
:1044A0009EA59B01AC010E94AE329B01AC01C801EC
:1044B000B7010E94F52E7B018C016FA178A589A51B
:1044C0009AA59B01AC010E94AE329B01AC01C801D0
:1044D000B7010E94F52E0E943B337B018C01A98D10
:1044E000BA8D5D966D937D938D939C93909760E0CC
:1044F00070E080E89FE3A80197010E94D52F2B016F
:104500003C012496BFAD2497BB2359F423966CAD90
:104510007DAD8EAD9FAD2397A30192010E94AE3277
:104520000CC060E070E080E89FE323962CAD3DADC9
:104530004EAD5FAD23970E94D52F5B016C01C80182
:10454000B701A60195010E94AE3228966CAF7DAFEF
:104550008EAF9FAF2897E98DFA8D618B728B838B1D
:10456000948B65857685878590890E9470307B0164
:104570008C01A60195010E94AE320E94BB2F0E94C1
:104580004230A98DBA8DD7966D937D938D939C9370
:10459000DA972091DC063091DD064091DE065091DD
:1045A000DF062BA33CA34DA35EA3C801B701A30163
:1045B00092010E94AE322BA13CA14DA15EA10E94AE
:1045C000AE3220E030E84BE355E40E94D52F0E9444
:1045D000BB2F0E943D30A98DBA8D9B966D937D9324
:1045E0008D939C939E976FA578A989A99AA9A301F9
:1045F00092010E94AE326F8F78A389A39AA36BA514
:104600007CA58DA59EA5A30192010E94AE326B8F61
:104610007C8F8D8F9E8F6FA178A589A59AA5A30108
:1046200092010E94AE321B012C0190919D05809158
:104630009E05981709F4B7C06090B8057090B90549
:104640008090BA059090BB05B301C40120E030E032
:1046500040E050E00E94DC3118160CF0A4C06091DC
:10466000AC057091AD058091AE059091AF05905865
:104670002F8D38A149A15AA10E94AE327B018C0135
:104680006B8D7C8D8D8D9E8D2091B0053091B10507
:104690004091B2055091B3050E94AE329B01AC012E
:1046A000C801B7010E94F42E7B018C01C201B10147
:1046B0002091B4053091B5054091B6055091B705EC
:1046C0000E94AE329B01AC01C801B7010E94F42EDA
:1046D0007B018C0123E333E343E75FE30E94CE2FAA
:1046E00088230CF060C0B301C40128962CAD3DAD09
:1046F0004EAD5FAD28970E94CE2F87FD08C028964B
:104700008CAD9DADAEADBFAD28973C014D01C8014C
:10471000B70123E333E343E75FEB0E94DC31181674
:104720000CF046C060E070E080E89FE3A8019701CC
:104730000E94F42E20E030E040E05FE30E94AE32C1
:104740000E943B335B016C016BA17CA18DA19EA1FA
:104750002091E0063091E1064091E2065091E30697
:104760000E94AE32A60195010E94AE327B018C01FF
:1047700060E070E080E89FE3A60195010E94F42EBE
:104780009B01AC01C801B7010E94D52F0E943B33A9
:104790007B018C01B301C4019701A8010E94CE2FB7
:1047A00087FD06C007C0EE24FF2400E010E002C031
:1047B00073018401C701D801E98DFA8D818F928F31
:1047C000A38FB48F6BA17CA18DA19EA1905820E0F6
:1047D00030E040E050EC0E94AE32A98DBA8D5D967B
:1047E0002D913D914D915C9190970E94AE3220E0C9
:1047F00030E040E050E00E94F52E0E943B33D62E80
:10480000C72EB82EA92EB701C8012D2D3C2D4B2D3A
:104810005A2D0E94CE2F87FD04C0ED2CFC2C0B2DB1
:104820001A2DC701D801E98DFA8D858B968BA78B40
:10483000B08F61897289838994892D2D3C2D4B2DF0
:104840005A2D0E94CE2F181634F081E0A98DBA8D12
:1048500092968C9303C0E98DFA8D12A281E0A98D06
:10486000BA8D91968C932D8A3E8A4F8A588E2B8DC5
:104870003C8D4D8D5E8D298B3A8B4B8B5C8B8F8D58
:1048800098A1A9A1BAA18D879E87AF87B88B64969E
:104890002CAD3DAD4EAD5FAD649729873A874B8710
:1048A0005C8760968CAD9DADAEADBFAD60978D83DE
:1048B0009E83AF83B8872C962CAD3DAD4EAD5FADDA
:1048C0002C9729833A834B835C83ACEAB5E0FE01E5
:1048D0003D968CE001900D928150E1F7E98DFA8DC3
:1048E00081899289A389B4898093B8059093B90589
:1048F000A093BA05B093BB0580919F0580939D0559
:1049000080919D058F5F823109F480E080939F053F
:10491000A0EAB5E0FE0131968CE001900D92815045
:10492000E1F70E943D1FCD5ADF4F0FB6F894DEBF6E
:104930000FBECDBFCF91DF911F910F91FF90EF90F0
:10494000DF90CF90BF90AF909F908F907F906F90AF
:104950005F904F903F902F9008951F931BE306C0E8
:104960000E949B128091BC05882391F490919D0533
:1049700080919E05981741F080919E05819FC0010E
:10498000112489589E4F61F78091BD05833041F312
:104990001F91089580919D0580939E0580919D05AE
:1049A0008F5F823109F480E080939F058CE1E0EA1B
:1049B000F5E0DF011D928A95E9F708956F927F92E5
:1049C0008F929F92AF92BF92CF92DF92EF92FF921F
:1049D0000F931F93CF93DF934C013B015A01FB01CF
:1049E0008081F401E80FF11DEF0189918D3229F4E6
:1049F00081812196CC24C39405C08B3211F481812E
:104A00002196CC2420E030E040E050E0DD24E0E0DE
:104A100070E0682F60536A30F8F4EF5FE930C0F45B
:104A20007111DA94DA01C901F2E0880F991FAA1F07
:104A3000BB1FFA95D1F7280F391F4A1F5B1F220FA2
:104A4000331F441F551F260F311D411D511D09C025
:104A5000772339F4D39405C06E3F29F4772319F4F2
:104A600071E08991D6CFEE2319F420E030E051C0F7
:104A7000CA01B9010E946E307B018C0120E030E058
:104A800040E050E00E94CE2F882369F42BC0C8017B
:104A9000B7012AE037ED43E25CE30E94AE327B01CE
:104AA0008C01F2E0DF0E8FEFD8168CF3D81659F494
:104AB000C801B7012DEC3CEC4CEC5DE30E94AE323A
:104AC0007B018C010FC0DD2069F0C801B70120E037
:104AD00030E040E251E40E94AE327B018C01DA9476
:104AE0001D149CF3CC2049F0D801C701B058F50142
:104AF00080839183A283B38305C0F501E082F182B4
:104B000002831383882D80958C0FF301808321E02D
:104B100030E0C901DF91CF911F910F91FF90EF908D
:104B2000DF90CF90BF90AF909F908F907F906F90CD
:104B3000089520EA3FE004C0F9013197F1F70197A9
:104B40000097D1F708951F93A0EABFE040E951E034
:104B500015E335E031C06A3071058105910540F4F7
:104B6000232F2A95F1F7615070408040904024C077
:104B7000643671058105910540F4212F2A95F1F7DE
:104B80006A5070408040904017C0683E23E0720732
:104B900020E0820720E0920740F4FA013197F1F714
:104BA000645670408040904007C0FD013197F1F796
:104BB000685E7340804090406115710581059105E4
:104BC00051F61F910895EF92FF920F931F936091FA
:104BD000BF057091C0058091C1059091C2052091DB
:104BE000C3053091C4054091C5055091C605E090BC
:104BF000C705F090C8050091C9051091CA050E942B
:104C00003B1D6091BF057091C0058091C1059091D9
:104C1000C2052091C3053091C4054091C50550914E
:104C2000C605E090C705F090C8050091C905109130
:104C3000CA050E9499081F910F91FF90EF90089567
:104C400084B1817F84B985B18E6085B98091E40695
:104C500083FF09C080916B008E6080936B00809110
:104C60006800816008C080916B00817F80936B0039
:104C7000809168008E7F8093680008952F923F9204
:104C80004F925F926F927F928F929F92AF92BF925C
:104C9000CF92DF92EF92FF920F931F93DF93CF9308
:104CA000CDB7DEB7A9970FB6F894DEBF0FBECDBF64
:104CB0008EA36FA348A738014901FE0131968CE00D
:104CC000DF011D928A95E9F70EA100FD02C010E0F8
:104CD0000FC06091C1067091C2068091C306909189
:104CE000C4060E947E3269837A838B839C8311E0A1
:104CF00001FF0FC01F5F6091C5067091C6068091CD
:104D0000C7069091C8060E947E326D837E838F8392
:104D1000988702FF0FC01F5F6091C9067091CA0695
:104D20008091CB069091CC060E947E3269877A876B
:104D30008B879C8789859A85AB85BC852D803E8035
:104D40004F805884281639064A065B0610F41C0169
:104D50002D0189819A81AB81BC81281639064A06CA
:104D60005B0610F41C012D01612F70E080E090E0E3
:104D70000E946E300E943B335B016C01C201B101A5
:104D80000E946E30A60195010E94D52F7B018C01F7
:104D90002091DC063091DD064091DE065091DF0661
:104DA0000E94AE3220E030E84BE355E40E94D52F5C
:104DB0000E94BB2F0E9442306AA37BA38CA39DA3B9
:104DC000C401B301A60195010E94AE329B01AC0162
:104DD000C801B7010E94AE329B01AC0160EC71EEDC
:104DE00084E69CE40E94D52F0E947E327B018C01D8
:104DF000B8EFEB16B4E2FB06B1E00B07B0E01B071F
:104E000018F45701680107C038EFA32E34E2B32E1F
:104E100031E0C32ED12C2091E506207E8091D7066B
:104E2000282729A33FA1332319F480EE282729A39B
:104E3000D201C101B695A7959795879566247724E9
:104E40004301681A790A8A0A9B0A8091CE06B60144
:104E5000A501481B5109610971094D8B5E8B6F8B50
:104E6000788F6D8E7E8E8F8E98A2698E7A8E8B8EC5
:104E70009C8E198A1A8A1B8A1C8A60E177E280E07C
:104E800090E06D877E878F87988B74E089A1872754
:104E900089A733B198A5992311F0AEE03A27BEA1B6
:104EA000B0FF1AC089819A81AB81BC81680E791EDE
:104EB0008A1E9B1E16141704180419046CF431FF83
:104EC00002C029A504C02EA12E7F2EA329A16218FD
:104ED00073088408950801C029A14EA141FF29C08B
:104EE0008D819E81AF81B8854D8D5E8D6F8D78A14E
:104EF000480F591F6A1F7B1F4D8F5E8F6F8F78A3DE
:104F00001416150616061706A4F432FF03C058E05F
:104F1000252703C06EA16D7F6EA38D8D9E8DAF8DF5
:104F2000B8A182199309A409B5098D8F9E8FAF8FFF
:104F3000B8A39EA192FF29C089859A85AB85BC85BF
:104F4000498D5A8D6B8D7C8D480F591F6A1F7B1FB1
:104F5000498F5A8F6B8F7C8F14161506160617060D
:104F6000C4F433FF03C050E1252703C06EA16B7F5B
:104F70006EA3898D9A8DAB8DBC8D82199309A4097E
:104F8000B509898F9A8FAB8FBC8F9EA1992309F4A5
:104F90006DC08091BE0584FD69C08BB12C71837E8C
:104FA000282B2BB96091CE0670E080E090E00E9443
:104FB000A325A9A1ABB96D897E898F89988D0E949F
:104FC000A325EA14FB040C051D0508F062CF2D850E
:104FD0003E854F8558892A0D3B1D4C1D5D1D2D8733
:104FE0003E874F87588B21326EE4360760E04607D4
:104FF00060E0560708F44DCF20523E4440405040F8
:105000002D873E874F87588B89899A89AB89BC89C0
:105010002AA13BA14CA15DA1820F931FA41FB51F24
:10502000898B9A8BAB8BBC8B60E077E883E993E04C
:1050300029893A894B895C890E94C633C901DA0102
:105040005C016D01AE14BF04C006D10610F4570117
:1050500068018091CE06B601A501481B510961097E
:1050600071094D8B5E8B6F8B788F13CFA9960FB61E
:10507000F894DEBF0FBECDBFCF91DF911F910F918E
:10508000FF90EF90DF90CF90BF90AF909F908F9068
:105090007F906F905F904F903F902F900895FF9278
:1050A0000F931F930E94CE140091EA061091EB0615
:1050B0002091EC063091ED0684E061E040E00E9432
:1050C0003E260091EA061091EB062091EC06309105
:1050D000ED0683E061E040E00E943E268091EE060E
:1050E0009091EF060E94992542E0F42EFA940091E7
:1050F000E6061091E7062091E8063091E90687E080
:1051000060E041E00E943E268091EE069091EF061D
:105110000E94992581E0F816A1F40091E60610910D
:10512000E7062091E8063091E90687E061E040E07B
:105130000E943E268091EE069091EF060E949925EE
:10514000D5CFFF2099F60E94D8151F910F91FF909F
:1051500008951F920F920FB60F9211242F933F9331
:105160004F935F936F937F938F939F93AF93BF936F
:10517000EF93FF938091BD05863059F08091BE0575
:1051800085FD07C00E9400048091BE058064809365
:10519000BE05FF91EF91BF91AF919F918F917F914C
:1051A0006F915F914F913F912F910F900FBE0F9094
:1051B0001F9018958F929F92AF92BF92CF92DF92DD
:1051C000EF92FF920F931F93DF93CF93CDB7DEB78C
:1051D0002A970FB6F894DEBF0FBECDBF7B018C01BE
:1051E00020E030E040E050E00E94CE2F88233CF4E5
:1051F0008DE20E94AB1117FB109517F91095A09046
:10520000F506DA2C0CC0C801B70120E030E048EC0C
:1052100052E40E94AE327B018C018EEFD80EE1E0A9
:10522000ED1588F3A0FE0AC0C801B70120E030E008
:1052300040E251E40E94AE327B018C01C801B7010B
:1052400020E030E040E05FE30E94F52E0E943D3018
:105250006B017C019E012F5F3F4FF901EA0DF11DAB
:105260008EE28083BB2449011EC0BA1409F4B394B2
:1052700084010B0D111DC701B6012AE030E040E0AA
:1052800050E00E94C633605DF8016083B394C701AB
:10529000B6012AE030E040E050E00E94C633C90188
:1052A000DA016C017D01C114D104E104F104E9F6D5
:1052B00006C0FC01EB0DF11D2083B39403C0CE01A9
:1052C000019620E3BA14A8F3BA1489F48B2D8F5FEA
:1052D000FE01E80FF11D90E39183B82EB39407C04F
:1052E000FE01EB0DF11D80810E94AB11BA94BB2031
:1052F000B9F72A960FB6F894DEBF0FBECDBFCF9197
:10530000DF911F910F91FF90EF90DF90CF90BF90B2
:10531000AF909F908F9008958F929F92BF92CF925F
:10532000DF92EF92FF920F931F93DF93CF93CDB74E
:10533000DEB72A970FB6F894DEBF0FBECDBF7B0154
:105340008C0197FF0BC08DE20E94AB111095009568
:10535000F094E094E11CF11C011D111D670178011E
:10536000C114D104E104F10421F480E30E94AB11E3
:105370002FC0BB244E010894811C911C84010B0D8D
:10538000111DC701B6012AE030E040E050E00E9464
:10539000C633605DF8016083B394C701B6012AE0AB
:1053A00030E040E050E00E94C633C901DA016C01F0
:1053B0007D01C114D104E104F10401F707C0FE012D
:1053C000EB0DF11D80810E94AB11BA94BB20B9F79F
:1053D0002A960FB6F894DEBF0FBECDBFCF91DF91F6
:1053E0001F910F91FF90EF90DF90CF90BF909F9013
:1053F0008F9008950F931F93DF93CF93CDB7DEB7B0
:1054000028970FB6F894DEBF0FBECDBF982FFE01D0
:1054100031969E01275F3F4F892F8170819396952A
:10542000E217F307C9F78E01085F1F4FF80180816B
:10543000805D0E94AB11015010400C171D07B1F7A1
:1054400028960FB6F894DEBF0FBECDBFCF91DF9187
:105450001F910F910895CF93DF93EC0102C00E943A
:10546000AB11FE01219684918823C9F7DF91CF917A
:105470000895CF93DF93EC0103C021960E94AB11F6
:1054800088818823D1F7DF91CF9108958AE594E050
:105490000E942B2A089588E895E00E942B2A0895FF
:1054A0001F93182F82EF95E00E942B2A133091F062
:1054B000143028F4113041F01230B1F408C0143027
:1054C00061F0153089F40CC080EE95E00BC08CECD7
:1054D00095E008C08AEB95E005C082EB95E002C03C
:1054E00089EA95E00E942B2A85EA95E00E942B2A02
:1054F0001F9108951F93182F882319F48BE197E0CB
:1055000050C083E197E00E942B2A173091F11830A8
:1055100070F4133011F1143028F41130C1F012304E
:10552000F1F518C01530F9F0163000F519C01A3031
:1055300049F11B3028F41830F9F0193081F51FC0FB
:105540001C3031F11C3008F11D3049F524C081E0D8
:1055500097E023C089EE96E020C083ED96E01DC061
:1055600084EC96E01AC08EEA96E017C08CE996E0CB
:1055700014C08BE896E011C08FE796E00EC080E77C
:1055800096E00BC08FE496E008C080E496E005C08A
:1055900085E396E002C087E296E00E942B2A84E22F
:1055A00096E00E942B2A1F910895AF92BF92CF924E
:1055B000DF92EF92FF920F931F93DF93CF93CDB7BC
:1055C000DEB768970FB6F894DEBF0FBECDBFDE0121
:1055D0001196EFEBF5E08CE001900D928150E1F730
:1055E0008091BD058430C9F0853038F4823079F07F
:1055F000833080F4882341F01DC08630A1F08630CE
:1056000078F08730B9F412C08CE191E011C085E1E7
:1056100091E00EC080E191E00BC08AE091E008C00B
:1056200084E091E005C08DEF90E002C086EF90E04D
:105630000E942B2A8FEE90E00E942B2A8DE0E82E0C
:10564000F12CEC0EFD1E670100E010E05E010894F5
:10565000A11CB11CF501E00FF11F608171818281F5
:1056600093810E947030F801EF53F94F208131810E
:10567000428153810E94D52F9B01AC01F6016083CA
:105680007183828393838091E40680FF0DC0CA01F9
:10569000B9012BE832E441E25DE30E94AE32F6014B
:1056A0006083718382839383F6016191719181910B
:1056B00091916F010E94DA288DEE90E00E942B2AD2
:1056C0000C5F1F4F0C30110529F687EE90E00E9409
:1056D0002B2A09EE15E0DD248091E40680FF1BC033
:1056E000F8016081718182819381248535854685A9
:1056F00057850E94F52E2BE832E441E25DEB0E94D3
:10570000AE329B01AC01F70160817181828193818E
:105710000E94F52E14C0F80160817181828193810D
:1057200024853585468557850E94F52E9B01AC0161
:10573000F70160817181828193810E94F42EF701CB
:105740006083718382839383F70160817181828199
:1057500093810E94DA28F2E0DF1621F085EE90E0D6
:105760000E942B2AD39484E090E0E80EF91E0C5F8F
:105770001F4F93E0D91609F0AFCF81EE90E00E9461
:105780002B2A68960FB6F894DEBF0FBECDBFCF911F
:10579000DF911F910F91FF90EF90DF90CF90BF901E
:1057A000AF9008958091CD05823091F0833028F438
:1057B000882341F08130B1F408C0833061F0843037
:1057C00089F40CC085E991E00BC081E991E008C043
:1057D0008DE891E005C089E891E002C084E891E09D
:1057E0000E942B2A81E891E00E942B2A6091E80513
:1057F00070E06A5C7F4F882777FD8095982F0E9424
:105800008C298091E505882319F0823039F403C092
:105810008CE791E005C087E791E002C082E791E064
:105820000E942B2A8091CF05882319F08DE691E004
:1058300002C088E691E00E942B2A8091D00588233F
:1058400019F083E691E002C08EE591E00E942B2AD8
:105850008091CE05882319F089E591E002C084E5A6
:1058600091E00E942B2A8091D105813041F0813056
:1058700018F0823059F406C080E591E005C08CE450
:1058800091E002C088E491E00E942B2A8091D20529
:10589000882359F0813019F08F3F59F403C084E414
:1058A00091E005C080E491E002C08CE391E00E94A9
:1058B0002B2A8091D305882319F0813041F403C04D
:1058C00088E391E002C084E391E00E942B2A81E307
:1058D00091E00E942B2A6091E40570E080E090E066
:1058E0000E948C298EE291E00E942B2A8091CF05A4
:1058F000882379F06091D4057091D5058091D60503
:105900009091D7052BE832E441E25DE30E94AE328C
:1059100008C06091D4057091D5058091D60590910D
:10592000D7050E94DA288AE291E00E942B2A089586
:10593000CF92DF92EF92FF920F931F93E82E6B01AD
:1059400087E291E00E942B2AFF2400E010E0C801CA
:10595000B7010E948C2985E291E00E942B2AC601A2
:105960000E94392A82E291E00E942B2A1F910F9116
:10597000FF90EF90DF90CF900895CF92DF92EF925B
:10598000FF920F931F93DF93CF93CDB7DEB72C9782
:105990000FB6F894DEBF0FBECDBFFF246E01089492
:1059A000C11CD11C8F2DB6010E94801C882321F4BC
:1059B0008AE00E947A2A90C08BEC91E00E942B2A08
:1059C00083E0F816E9F08F1530F0E1E0FE1691F073
:1059D000EF1598F00CC0F5E0FF16C1F0FF1698F037
:1059E00086E0F816B1F0E7E0FE16D1F415C087ECBA
:1059F00091E014C083EC91E011C08FEB91E00EC0F8
:105A00008BEB91E00BC087EB91E008C083EB91E05A
:105A100005C08FEA91E002C08BEA91E00E942B2A38
:105A20008601EE248091E40680FF0CC0F8016081BD
:105A30007181828193812BE832E441E25DE30E942F
:105A4000AE3205C0F80160817181828193810E942C
:105A5000DA28F2E0EF1619F089EA91E002C085EA4F
:105A600091E00E942B2AE3940C5F1F4F83E0E8161D
:105A7000C9F6F394E8E0FE1609F094CF8FE991E0BF
:105A80000E942B2A05EF15E0FF248091E40680FF99
:105A90000CC0F80160817181828193812BE832E42E
:105AA00041E25DE30E94AE3205C0F8016081718180
:105AB000828193810E94DA28F2E0FF1619F08DE9C5
:105AC00091E002C089E991E00E942B2AF3940C5FD7
:105AD0001F4F83E0F816C9F62C960FB6F894DEBF78
:105AE0000FBECDBFCF91DF911F910F91FF90EF902F
:105AF000DF90CF90089586E594E00E942B2A609174
:105B0000C1067091C2068091C3069091C4060E949E
:105B1000DA2883E494E00E942B2A6091C5067091F4
:105B2000C6068091C7069091C8060E94DA2880E3D5
:105B300094E00E942B2A6091C9067091CA06809158
:105B4000CB069091CC060E94DA288DE194E00E9469
:105B50002B2A6091CE0670E080E090E00E948C29B4
:105B600084E094E00E942B2A6091CF067091D006C9
:105B70008091D1069091D2060E94DA2887EE93E0B8
:105B80000E942B2A6091D3067091D4068091D5068D
:105B90009091D6060E94DA288AEC93E00E942B2A84
:105BA0006091D70670E080E090E00E948C298CEA3A
:105BB00093E00E942B2A8091D7060E94FA2985EA59
:105BC00093E00E942B2A6091F40670E080E090E060
:105BD0000E948C2987E893E00E942B2A6091DC06C2
:105BE0007091DD068091DE069091DF0620E030E0C6
:105BF00041E655E40E94D52F0E94DA2888E693E01A
:105C00000E942B2A6091E0067091E1068091E206E5
:105C10009091E3060E94DA2888E493E00E942B2A00
:105C20006091D8067091D9068091DA069091DB06D2
:105C30000E94DA288FE293E00E942B2A6091F606F8
:105C400070E080E090E00E948C2980E193E00E9467
:105C50002B2A6091F50670E080E090E00E948C298C
:105C600087EF92E00E942B2A6091E40670E080E0CA
:105C700090E061707070807090700E948C298AED45
:105C800092E00E942B2A6091E40670E07695679579
:105C900080E090E061707070807090700E948C293C
:105CA00080EC92E00E942B2A6091E40670E07695E9
:105CB00067957695679580E090E061707070807070
:105CC00090700E948C298EE992E00E942B2A6091AC
:105CD000E40670E023E0769567952A95E1F780E089
:105CE00090E061707070807090700E948C2983E8E1
:105CF00092E00E942B2A6091E40670E094E0769591
:105D000067959A95E1F780E090E06170707080701F
:105D100090700E948C2987E692E00E942B2A609165
:105D2000E50670E080E090E00E948C2988E492E033
:105D30000E942B2A8091E5060E94FA2980E492E0D5
:105D40000E942B2A6091E6067091E7068091E80692
:105D50009091E9060E94DA2883E292E00E942B2AC1
:105D60006091EA067091EB068091EC069091ED0649
:105D70000E94DA2886E092E00E942B2A6091EE06CB
:105D80007091EF0680E090E00E948C2987EE91E010
:105D90000E942B2A6091F0067091F1068091F20624
:105DA0009091F3060E94DA288EEC91E00E942B2A53
:105DB00008951F93182F8CE196E00E942B2A1E3F16
:105DC00029F01F3F39F481E196E002C08EEF95E0A3
:105DD0000E942B2A84EF95E00E942B2A84EF91E009
:105DE0000E9499251F9108955058BB27AA270ED0CD
:105DF00081C241D230F046D220F031F49F3F11F4FD
:105E00001EF411C20EF4E095E7FBDCC1E92F94D239
:105E100080F3BA17620773078407950718F071F4C7
:105E20009EF5C3C20EF4E0950B2EBA2FA02D0B01E8
:105E3000B90190010C01CA01A0011124FF27591BCF
:105E400099F0593F50F4503E68F11A16F040A22FD5
:105E5000232F342F4427585FF3CF46953795279546
:105E6000A795F0405395C9F77EF41F16BA0B620B45
:105E7000730B840BBAF09150A1F0FF0FBB1F661F8C
:105E8000771F881FC2F70EC0BA0F621F731F841FCF
:105E900048F4879577956795B795F7959E3F08F0F5
:105EA000B3CF9395880F08F09927EE0F97958795B4
:105EB0000895E1D158F080E891E009F49EEFE2D135
:105EC00028F040E851E059F45EEF09C0ACC16DC262
:105ED000E92FE07831D268F3092E052AC1F326179D
:105EE00037074807590738F00E2E07F8E02569F004
:105EF000E025E0640AC0EF6307F8009407FADB01CD
:105F0000B9019D01DC01CA01AD01EF935DD0F2D171
:105F10000AD05F91552331F02BED3FE049E450FD6D
:105F200049EC63CF0895DF93DD27B92FBF7740E8B1
:105F30005FE31616170648075B0710F4D92FA1D2A6
:105F40009F938F937F936F93E0D3E6E9F0E06ED158
:105F5000D1D12F913F914F915F910CD3DD2349F027
:105F60009058A2EA2AED3FE049EC5FE3D0785D2744
:105F70004DDFDF91BFC102D280F09F3740F4911115
:105F80000EF414C260E070E080E89FE3089526F00C
:105F90001B16611D711D811D1BC135C1EFD008F499
:105FA00081E0089577D1E395B6C10CD0A3C16AD141
:105FB00040F061D130F021F45F3F19F003C151117D
:105FC000F5C131C1B9D198F39923C9F35523B1F380
:105FD000951B550BBB27AA2762177307840738F058
:105FE0009F5F5F4F220F331F441FAA1FA9F333D0B7
:105FF0000E2E3AF0E0E830D091505040E695001C6B
:10600000CAF729D0FE2F27D0660F771F881FBB1F26
:10601000261737074807AB07B0E809F0BB0B802D00
:10602000BF01FF2793585F4F2AF09E3F510568F04C
:10603000C9C0BCC15F3FECF3983EDCF38695779511
:106040006795B795F7959F5FC9F7880F911D96954E
:10605000879597F90895E1E0660F771F881FBB1FAA
:10606000621773078407BA0720F0621B730B840B57
:10607000BA0BEE1F88F7E095089504D06894B1112B
:1060800095C1089561D188F09F5790F0B92F992755
:10609000B751A0F0D1F0660F771F881F991F1AF033
:1060A000BA95C9F712C0B13081F07FD1B1E008953F
:1060B0007CC1672F782F8827B85F39F0B93FCCF3C0
:1060C000869577956795B395D9F73EF49095809529
:1060D000709561957F4F8F4F9F4F0895E89409C049
:1060E00097FB3EF490958095709561957F4F8F4F0B
:1060F0009F4F9923A9F0F92F96E9BB279395F69521
:10610000879577956795B795F111F8CFFAF4BB0F9E
:1061100011F460FF1BC06F5F7F4F8F4F9F4F16C002
:10612000882311F096E911C0772321F09EE8872F8C
:10613000762F05C0662371F096E8862F70E060E048
:106140002AF09A95660F771F881FDAF7880F9695C1
:10615000879597F9089512D180F09F3740F49111F7
:106160000EF024C160E070E080E89FEB089526F413
:106170001B16611D711D811D2BC045C0990F0008A4
:10618000550FAA0BE0E8FEEF16161706E807F90709
:10619000C0F012161306E407F50798F0621B730BA4
:1061A000840B950B39F40A2661F0232B242B252B25
:1061B00021F408950A2609F4A140A6958FEF811DC8
:1061C000811D089597F99F6780E870E060E0089569
:1061D000882371F4772321F09850872B762F07C0FE
:1061E000662311F499270DC09051862B70E060E072
:1061F0002AF09A95660F771F881FDAF7880F969511
:10620000879597F908959F3F49F0915028F4869516
:1062100077956795B7959F5F80389F4F880F9695C4
:10622000879597F908959FEF80EC0895DF93CF93BA
:106230001F930F93FF92EF92DF927B018C01689482
:1062400005C0DA2EEF0196D1FE01E894A5912591C3
:10625000359145915591AEF3EF01D8DDFE019701DF
:10626000A801DA9479F7DF90EF90FF900F911F91DA
:10627000CF91DF91089500240A9416161706180688
:106280000906089500240A9412161306140605063A
:106290000895C9CF59D0E8F3E894EFEFBB273FE06A
:1062A00048EC5FE76B3D73078407950708F1FF270C
:1062B0009F57B25A6A4D7F40894CF04032F4BE5528
:1062C0006542704F8643FF4F0894EE1F915030F0A7
:1062D000BB0F661F771F881FFF1FEBCF9EE788232A
:1062E00032F0BB0F661F771F881F9A95C1F79395F1
:1062F000E09589CF092E0394000C11F4882352F005
:10630000BB0F40F4BF2B11F460FF04C06F5F7F4FE1
:106310008F4F9F4F0895EF93E0FF06C0A2EA2AED4A
:106320003FE049EC5FEB72DDE5DF0F90039401FC89
:106330009058E3ECF0E0FAC157FD9058440F551F18
:1063400059F05F3F71F04795880F97FB991F61F0F7
:106350009F3F79F087950895121613061406551F6E
:10636000F2CF4695F1DF08C0161617061806991FDA
:10637000F1CF86957105610508940895E5DFA0F0D9
:10638000BEE7B91788F4BB279F3860F41616B11D15
:10639000672F782F8827985FF7CF86957795679531
:1063A000B11D93959639C8F30895E894BB276627E5
:1063B0007727CB0197F90895E1DE08F48FEF089570
:1063C0005ADF19F05FDF09F02ECFFCCEB901CA0108
:1063D0001ACF9F775F77B0DF98F39923B9F35523EE
:1063E000B9F3FF27951758F4E52FE91BED3070F747
:1063F0005E3B10F0F1E41CC09034E0F40AC0E92FD9
:10640000E51BED3028F79E3B10F0F1E411C050344D
:1064100088F4F9EA88232AF09A95660F771F881F77
:10642000DAF744232AF05A95220F331F441FDAF774
:106430009F1B5F1BFF931F930F93FF92EF927901B6
:106440008A01BB27AB2F9B01AC0196D09701A80115
:10645000BF937B018C01AA27BA2FB901CA018CD046
:10646000AF919701A801EF90FF900F911F91CEDCA3
:1064700041DF01D14F9140FF0895552747FD5095C9
:1064800009C09B01AC0160E070E080E89FE38DCD26
:1064900099CEB9CE59DFE8F39923D9F3940F511D62
:1064A000BBF39150504094F059F0882332F0660FBE
:1064B000771F881F91505040C1F79E3F510544F708
:1064C000880F911D9695879597F908955F3FACF0D9
:1064D000983E9CF0BB27869577956795B79508F40D
:1064E000B1609395C1F7BB0F58F711F460FFE8CF87
:1064F0006F5F7F4F8F4F9F4FE3CF58CF25DF58F10E
:106500009E5758F19851A0F0E9F0983020F5092EE7
:106510009927660F771F881F991F0A94D1F712C019
:10652000062E672F782F8827985F11F4000C07C07C
:10653000993FB4F38695779567959395D9F7611D43
:10654000711D811D3EF490958095709561957F4FEA
:106550008F4F9F4F0895689429CF27CF0BD0CACE75
:106560008ADE28F08FDE18F0952309F02BCE5BCE63
:1065700011241CCFE1DEA0F3959FD1F3950F50E0DD
:10658000551F629FF001729FBB27F00DB11D639FE5
:10659000AA27F00DB11DAA1F649F6627B00DA11D8B
:1065A000661F829F2227B00DA11D621F739FB00D31
:1065B000A11D621F839FA00D611D221F749F3327A1
:1065C000A00D611D231F849F600D211D822F762F3A
:1065D0006A2F11249F5750408AF0E1F088234AF037
:1065E000EE0FFF1FBB1F661F771F881F9150504083
:1065F000A9F79E3F510570F0E5CDD8CE5F3FECF393
:10660000983EDCF3869577956795B795F795E7956E
:106610009F5FC1F7FE2B880F911D9695879597F97F
:10662000089592DEE0F09E37D8F09639B8F49E389F
:1066300048F4672F782F8827985FF9CF869577954C
:10664000679593959539D0F3B62FB1706B0F711D87
:10665000811D20F48795779567959395B9CDD3CD16
:10666000A5CE9F9317DE0F9007FCEE5F54CE11F47A
:106670000EF4D9CDC8CD68DED0F39923D9F3CEF38B
:106680009F57550B87FF4BD056959795B0E020F458
:10669000660F771F881FBB1F1F930F930024900165
:1066A000A0018001F001A0E80E0F1F1F0A1E511D5E
:1066B000601B710B8009B50B48F4600F711F801DC2
:1066C000B51F0E1B1F0B0A0A510907C02E0F3F1FD3
:1066D0004A1F0E0F1F1F0A1E511D660F771F881FAE
:1066E000BB1FA695F795E795F8F606171707080656
:1066F0005B07211D311D411D0F911F91B901842F91
:106700009158880F9695879508959B01AC0126CFE7
:1067100035DE20F09F3708F449CE5ACD74CD915024
:106720005040660F771F881FD2F708959F938F936D
:106730007F936F93FF93EF939B01AC010FDFEF917A
:10674000FF9174DD2F913F914F915F9107CF629F31
:10675000D001739FF001829FE00DF11D649FE00D59
:10676000F11D929FF00D839FF00D749FF00D659FBA
:10677000F00D9927729FB00DE11DF91F639FB00DB9
:10678000E11DF91FBD01CF0111240895A1E21A2EC8
:10679000AA1BBB1BFD010DC0AA1FBB1FEE1FFF1FC5
:1067A000A217B307E407F50720F0A21BB30BE40B15
:1067B000F50B661F771F881F991F1A9469F760955C
:1067C0007095809590959B01AC01BD01CF01089516
:0467D000F894FFCF6B
:00000001FF
